:1000000000FCFF1F11040000A11E0000310F0000C2
:10001000310F0000310F0000310F0000310F0000E0
:10002000310F0000310F0000310F0000310F0000D0
:10003000310F0000310F0000310F0000112D0000C2
:10004000310F0000310F0000310F0000310F0000B0
:10005000310F0000310F0000310F0000310F0000A0
:10006000310F0000310F0000310F0000310F000090
:10007000310F0000310F0000310F0000310F000080
:10008000310F0000310F0000310F0000310F000070
:10009000310F0000310F0000310F0000310F000060
:1000A000512E0000310F0000310F0000310F000011
:1000B00071780000310F0000310F0000310F000097
:10040000FFFFFFFFFFFFFFFFFFFFFFFF7EFFFFFF7D
:1004100072B6244880F30888234880F309880220B4
:1004200080F31488BFF36F8F00F042FD03F0C8F82B
:100430001E481F491B4A914202DA08600431FAE75C
:100440001C49194A914202DA08600431FAE71A4954
:100450001A4A1B4B9A4204DA0868106004310432CD
:10046000F8E700201749184A914202DA086004317F
:10047000FAE700F035FD00F023FD144C144DAC42BA
:1004800003DA216888470434F9E703F059FD114C79
:10049000114DAC4203DA216888470434F9E70F496B
:1004A0000847000000FCFF1F00FEFF1F5555555573
:1004B00000F8FF1F00FCFF1FCC92000000FEFF1F92
:1004C00040FEFF1F00000020280C00201004000048
:1004D000100400001004000010040000D10E000001
:1004E000F0B544464D4656465F46F0B46B46CB6089
:1004F000C3689D46F0BCA046A946B246BB46F0BDC7
:1005000000F0C6FD62B6281CA047002001F0B0F93B
:1005100000F0A6FD01F03CF800F0BAFD014A024BE4
:100520001360FEE704ED00E0000000800000000022
:10053000002243088B4274D303098B425FD3030A22
:100540008B4244D3030B8B4228D3030C8B420DD335
:10055000FF22090212BA030C8B4202D312120902C3
:1005600065D0030B8B4219D300E0090AC30B8B4201
:1005700001D3CB03C01A5241830B8B4201D38B03AF
:10058000C01A5241430B8B4201D34B03C01A524154
:10059000030B8B4201D30B03C01A5241C30A8B4297
:1005A00001D3CB02C01A5241830A8B4201D38B0282
:1005B000C01A5241430A8B4201D34B02C01A524126
:1005C000030A8B4201D30B02C01A5241CDD2C30998
:1005D0008B4201D3CB01C01A524183098B4201D314
:1005E0008B01C01A524143098B4201D34B01C01AFF
:1005F000524103098B4201D30B01C01A5241C30877
:100600008B4201D3CB00C01A524183088B4201D3E5
:100610008B00C01A524143088B4201D34B00C01AD1
:100620005241411A00D20146524110467047FFE73D
:1006300001B5002000F0FCF802BDC0460029F7D04B
:1006400003B5FFF775FF0EBC4243891A1847C04631
:1006500003460B437FD4002243088B4274D3030923
:100660008B425FD3030A8B4244D3030B8B4228D3C4
:10067000030C8B420DD3FF22090212BA030C8B42EA
:1006800002D31212090265D0030B8B4219D300E08A
:10069000090AC30B8B4201D3CB03C01A5241830B0F
:1006A0008B4201D38B03C01A5241430B8B4201D3BF
:1006B0004B03C01A5241030B8B4201D30B03C01AE8
:1006C0005241C30A8B4201D3CB02C01A5241830A62
:1006D0008B4201D38B02C01A5241430A8B4201D391
:1006E0004B02C01A5241030A8B4201D30B02C01ABB
:1006F0005241CDD2C3098B4201D3CB01C01A524122
:1007000083098B4201D38B01C01A524143098B42AA
:1007100001D34B01C01A524103098B4201D30B0193
:10072000C01A5241C3088B4201D3CB00C01A5241B8
:1007300083088B4201D38B00C01A524143088B427D
:1007400001D34B00C01A5241411A00D20146524116
:10075000104670475DE0CA0F00D04942031000D335
:100760004042534000229C4603098B422DD3030A8A
:100770008B4212D3FC22890112BA030A8B420CD39A
:10078000890192118B4208D3890192118B4204D3C3
:1007900089013AD0921100E08909C3098B4201D343
:1007A000CB01C01A524183098B4201D38B01C01A7D
:1007B000524143098B4201D34B01C01A52410309F4
:1007C0008B4201D30B01C01A5241C3088B4201D3A3
:1007D000CB00C01A524183088B4201D38B00C01A50
:1007E0005241D9D243088B4201D34B00C01A524127
:1007F000411A00D20146634652415B10104601D3B4
:100800004042002B00D54942704763465B1000D33D
:10081000404201B5002000F00BF802BD0029F8D0DD
:1008200003B5FFF715FF0EBC4243891A1847C046AF
:100830007047C046000000000000000000000000FB
:10084000F0B55F4656464D464446F0B4051C061CBE
:10085000080387B099464F00030BCC0F92469B4686
:100860007F0D019467D06C4B9F4236D080205B4651
:1008700040031843C0006B0F1843684B83469C46E7
:1008800000239846EE00674400934B4649461D03FB
:10089000C90F5B0052462D0B5B0D894600D16EE0FF
:1008A0005D498B4264D080205C4940038C46002126
:1008B0000543ED00500F0543D20063444846FF183E
:1008C0007B1C9A46009B604002900B430F2B00D983
:1008D000ACE053489B00C3589F465B461D4300D085
:1008E00082E00823009300239B46023300269846AB
:1008F000CBE7029B01934346022B59D101240025EB
:100900000026019B1C40444B00212D030A0D1205BB
:100910002D0B1543434A1B0515401D436D00E4078D
:100920006D082543301C291C07B03CBC90469946F5
:10093000A246AB46F0BD2B434ED05B46002B00D108
:1009400085E1584600F094FA021C2823291C9B1AC2
:10095000161C5846D940083EB0400B1CB540034316
:100960009B462E1C0023304F0093BF1A98468CE7FD
:10097000514629432ED10025002202219EE75146EF
:10098000294323D0002D00D154E1281C00F070FA37
:10099000031C28215046C91A1A1CC8405146083A5F
:1009A000914095400A1C05431F480021C31A85E762
:1009B000032B00D1C2E1012B00D06DE14446019B25
:1009C00000251C40E4B2002300269DE700250022FC
:1009D000012173E7032171E70423009300239B4661
:1009E00001330026984650E70C230093093B9846B4
:1009F0004BE7802500242D030026074B84E74B4658
:100A0000AB46161C0193884675E7029BAB46161C45
:100A1000019388466FE7C046FF07000001FCFFFF17
:100A20008C7A0000FFFF0F800DFCFFFF330C3604B3
:100A3000360C9C46331C140C1204120C534398467B
:100A4000634653439946634663430193331C4146CF
:100A50006343090C4B445B18994505D9802040023B
:100A60008146019949440191190C039141460904B9
:100A7000090C1B045B1804932B0C9846331C2D04A3
:100A8000290C4B43604600934346654658435E43FA
:100A9000009B4D431B0C9946AE194E448446B5420B
:100AA00003D980235B029946CC44350C2B1C039858
:100AB000634484460593009B36041B041B0CF31807
:100AC0009C446046039058460504060C280C844656
:100AD0005043351C81466046654344434846000CFC
:100AE0008346724314195C44A24203D98022520205
:100AF00093465D44220CAD184A461204120C24049D
:100B00004046A41862464A437143464360460096F5
:100B1000464670438046100C84468844E044414574
:100B200005D9802149028C460099614400910198C1
:100B300003998446614499429B415B4299460598DA
:100B4000434684461204120C1B049B1863449C46C3
:100B5000AB4683429B4140460A19CC44A24289419C
:100B6000E344CC45B6415C46000C8046494276429F
:100B70005B426418334398448C428941AB459B41A6
:100B800049425B4219430D1C009B4544EE18760216
:100B9000E50D2E43B346049B56021E43731E9E4131
:100BA0005B46D20D324366021643DB010AD50123B0
:100BB000334076081E435B46DB071E435B465B08FB
:100BC0009B465746634BFB18002B5ADD720709D032
:100BD0000F223240042A05D0321DB242B64176427D
:100BE000B344161C5A46D20106D55A465A4B1A40EF
:100BF00080239346DB00FB18584A934234DD0124DE
:100C0000029B00251C400026554B7DE680205B465C
:100C10000003034208D0054206D105432D032D0BE6
:100C20004C46161C4E4B6FE65D4605432D032D0BBF
:100C30004B4B69E6504600F01BF9031C2033272B71
:100C400000DCA6E65546083885400022ACE6281CA4
:100C500000F00EF9021C2032272A00DC75E6083865
:100C600085400026AB467DE65A46F60852071643F5
:100C70005A4601245502029A5B052D0B5B0D144068
:100C800042E6384DED1B382D0ADD0124029B00257C
:100C90001C400026002337E6019B5746029391E74C
:100CA0001F2D25DC304B321C9C466744BE405B4602
:100CB000BB40371CEA407E1EB74113433B431E1C1A
:100CC0005B46EB401D1C730709D00F233340042BF8
:100CD00005D0331DB342B6417642AD191E1C2B021E
:100CE00020D50124029B00251C40002601230BE691
:100CF0005A461E4BDB1BDA40131C202D1CD01C4A0D
:100D000094465A466744BA40171C3E43721E9641A9
:100D10001E4307230025334007D00F23002533400F
:100D2000042BD6D16B076D022D0B0124F6081E4350
:100D3000029B1C400023E7E50027E6E780255B4691
:100D400001242D031D43019B2D0323401C1C2D0B4F
:100D5000034BD9E5FF030000FFFFFFFEFE07000085
:100D6000FF07000002FCFFFF1E040000E2FBFFFF84
:100D70003E04000000000000000000000000000031
:100D80000B0330B5134C1A0B4B00051C5B0DC90F40
:100D90000020A34210DD104883420EDC80200F4C5F
:100DA00040030243E41A1F2C0ADD0D48C31ADA403F
:100DB000131C48424340581830BD0A4BC818FBE783
:100DC000281CE040084CA44663449A40131C03438B
:100DD000EFE7C046FE0300001D04000033040000DE
:100DE00013040000FFFFFF7FEDFBFFFF000000008A
:100DF00038B5041E16D0C50F00D04442201C00F0A8
:100E000037F8174B1B1A0A2821DC021C211C15324B
:100E100091400A1C0B21081AC4405B052403240BD3
:100E20005B0D03E000250023002400220021101C9C
:100E300024030A0D1205240B14430A4A1B0514400F
:100E40001C436400ED0764082C43211C38BD0B389B
:100E500084405B052403240B5B0D0022E6E7C046BB
:100E60001E040000FFFF0F800000000000000000D3
:100E70001C2101231B04984201D3000C10391B0ACA
:100E8000984201D3000A08391B09984201D300098E
:100E9000043902A2105C40187047C04604030202E5
:100EA000010101010000000000000000000000003E
:100EB0007047C04600000000000000000000000075
:100EC0007047C04600000000000000000000000065
:100ED000FEE7C04600000000000000000000000027
:100EE000F0B50F4E0025371C80377368B468316841
:100EF000A3420AD21A1C01C901C2A242FBD3DA439F
:100F00001419A4080134A4001B19F268934202D2F8
:100F100020C39342FCD31036BE42E6D3F0BDC04698
:100F2000CC7A00000000000000000000000000007B
:100F3000FEE7C046000000000000000000000000C6
:100F400030BFFDE7000000000000000000000000CE
:100F500010B500F0ADF900F043F900230F4C236306
:100F6000636300F095FE00F0EBFE201C0C4980222C
:100F7000383000F03DFB0B4B0122C3612023C254EB
:100F8000094A0A4B116AA0610B40136200F058F83D
:100F900062B6074800F0ACFB10BDC046D800002088
:100FA000CC7C000000FCFF1F00ED00E0FFFF00FF15
:100FB0004C7B00000000000000000000000000006A
:100FC00072B6014BD862FEE7D80000200000000096
:100FD000F0B5474680B400F0D3F82322154DA96937
:100FE0008B5C002B01D0013B8B542F1C00F0C8F808
:100FF000AB6AEC6901331C37AB62BC4217D0A36803
:10100000013BA360002B12D198464346E668E3609B
:1010100023685F60EB6100F06BF862B62069B0474F
:1010200072B600F04DF8EC69A368002BEDD004BC5B
:101030009046F0BDD8000020000000000000000035
:1010400008B5054B1A6B002A02D15B6B002B02D04E
:101050000248FFF7B5FF08BDD80000207C7B0000E8
:1010600010B5064C236B002B02D1636B002B02D012
:101070000348FFF7A5FF0123636310BDD8000020DC
:10108000847B000000000000000000000000000061
:1010900010B5074C236B002B05D1636B002B02DDD1
:1010A0000023636310BD0348FFF78AFFF8E7C046DB
:1010B000D80000208C7B0000000000000000000031
:1010C00010B5064C236B002B02DD636B002B02D0A6
:1010D0000348FFF775FF0123636310BDD8000020AC
:1010E000947B0000000000000000000000000000F1
:1010F00010B5074C236B002B05DD636B002B02DD65
:101100000023636310BD0348FFF75AFFF8E7C046AA
:10111000D80000209C7B00000000000000000000C0
:1011200010B572B6074C236B002B02DB626B002AF2
:1011300003D00548FFF744FF236B0133236362B6F6
:1011400010BDC046D8000020A47B000000000000B5
:1011500010B572B6074C236B002B02DD626B002AC0
:1011600003D00548FFF72CFF236B013B236362B6D6
:1011700010BDC046D8000020AC7B0000000000007D
:1011800008B5064B1A6B002A03DB5B6B002B00DDF6
:1011900008BD0348FFF714FFFAE7C046D800002057
:1011A000B47B000000000000000000000000000010
:1011B00008B5064B1A6B002A03D15B6B002B00DDD0
:1011C00008BD0348FFF7FCFEFAE7C046D800002040
:1011D000BC7B0000000000000000000000000000D8
:1011E000054B1A1C1C32DA611A62012252425A6201
:1011F00000229A627047C046D8000020000000001C
:10120000F8B5051C0C1C161C1F1CFFF7B9FF002DA0
:101210001CD0002E1AD0002C18D00E492F61CB699B
:10122000EE609A68944204D91B68A41A9A68A24294
:10123000FAD35A682B606A6015605D60AC609A688A
:10124000141B9C6001235B424B62F8BD0248FFF710
:10125000B7FEE2E7D8000020D47B000000000000C9
:1012600010B5041CFFF78CFF002C17D0E368002B8F
:1012700010D0A16823688C469A6862449A606268BC
:10128000136023685A6000230122E360054B524239
:101290005A6210BD0448FFF793FEEAE70248FFF7E1
:1012A0008FFEE3E7D8000020C47B000000000000B0
:1012B0000022034B1B605B609A601B615B6170479F
:1012C000D800002000000000000000000000000026
:1012D00010B5041CFFF754FF002C19D02023E35C49
:1012E000002B11D00F2B0FD000222023E254A26834
:1012F000094B1B6899689142FBD25A68236062606F
:10130000201C14605C6010BD0448FFF759FEEBE739
:101310000248FFF755FEE1E7D8000020347C0000CA
:1013200038B5041C72B6FFF7CBFE2023E35C072B15
:101330000ED8114A9B00D3589F46656AFFF720FFDD
:10134000AB680133AB60226863681A60226853603F
:1013500001235B426362201CFFF7BAFFFFF7C8FE60
:1013600062B638BD0022636A201C1A6001235B420A
:101370006362FFF7ADFFF1E7E07B000000000000D3
:1013800010B5041CFFF7FCFE002C19D02023E35CF1
:10139000002B11D00F2B0FD000222023E254A26883
:1013A000094B1B6899689142FBD85A6823606260B8
:1013B000201C14605C6010BD0448FFF701FEEBE7E1
:1013C0000248FFF7FDFDE1E7D8000020007C0000A7
:1013D00070B50F4C061CA569FFF7EAFE2023142107
:1013E00023222068EE54A95402685460226001222E
:1013F000A061C254EFF30983EA69243B9A4203D9FE
:101400000448FFF7DDFDA069291CFFF769F870BDEE
:10141000D8000020247C0000000000000000000034
:1014200070B50C1C86B0061CFFF7C2FE631C15D0FD
:101430000D4D211CAB690D4A01A8FFF7E1FE301CE0
:10144000FFF7C6FFFFF79CFE049B002B02D001A80C
:10145000FFF706FFAB69586A06B070BD301CFFF796
:10146000B7FF014DF6E7C046D80000202113000069
:10147000F8B5194C051C0F1CA669FFF799FE2368E7
:10148000A34204D0A2699B6892689A421BD3AB68BE
:10149000B2686F62934212D9301CFFF719FF012224
:1014A0002023061CA561EA54EFF30983C269243B9B
:1014B0009A420CD8281C311CFFF712F8F8BD281CE2
:1014C000FFF706FFFAE70548FFF77AFDDFE7044874
:1014D000FFF776FDEEE7C046D8000020147C000040
:1014E000247C00000000000000000000000000005C
:1014F0002320084B1A689B699168185C9A68002839
:1015000003D191424041C0B270478A42804140427B
:10151000FAE7C046D80000200000000000000000EC
:1015200038B50D4C01212368A0691A685460226007
:1015300020229954A361FFF723FF051CEFF30983D1
:10154000C269243B9A4202D90448FFF739FD291C9D
:10155000A069FEF7C5FF38BDD8000020247C00003C
:1015600008B5FFF725FEFFF70BFE054B1A689B69D0
:1015700092689B689A4201D9FFF7D2FF08BDC04626
:10158000D800002000000000000000000000000063
:1015900070B5124C01212368A0691A682326546093
:1015A00022602022A36199549B5D002B12D1FFF78A
:1015B0008FFE1423051C8355EFF30983EA69243B4E
:1015C0009A4202D90648FFF7FBFC291CA069FEF7E6
:1015D00087FF70BDFFF7D4FE051CEDE7D8000020A3
:1015E000247C00000000000000000000000000005B
:1015F00030B5022420238260C454002314251F34F4
:10160000035502340555C2630122836343632233C9
:10161000C254074B81615A6903614261106158618C
:10162000031C283383620433C362036330BDC046A6
:10163000D8000020000000000000000000000000B2
:1016400038B5041CFFF79CFD002C47D007236268C7
:101650001A4202D1A168194234D02248FFF7B0FCE7
:10166000E268FF2A34D82569002D31D0A36861686B
:10167000181C4838C161191C6C39C1600D6165695D
:101680004D61194D0D622168022481612021826023
:101690004454002114251F34015502340555C263FA
:1016A00022228163416301318154104A51690261F0
:1016B0004161086150611A1C1C3B203A12601B609A
:1016C0005B6038BD8A42C8D28A1AC72AC8D8C4E724
:1016D0000448FFF775FC2569E268C7E70148FFF792
:1016E0006FFCB3E7407C000001050000D80000203B
:1016F00010B5041C406800F0A3F9002802D013487C
:10170000FFF75EFCA26863685521934203D219700B
:1017100001339A42FBD172B6FFF7A2FC201CFFF7FF
:101720008FFF0021041CFFF7A3FEFFF7B1FC084B5D
:101730001A689A4207D09B6999689368994202D2C5
:101740000448FFF73DFC62B6201C10BD587C000029
:10175000D8000020947C0000000000000000000081
:1017600038B5041C72B62225FFF77AFC635D002BA6
:1017700018D02222013BA354226A234B13400F2B83
:101780001CD0FFF785FC214B1A689A4204D09B6954
:1017900099689368994201D362B638BD1C48FFF737
:1017A0000FFCF9E71B48FFF70BFC2222635D013BAE
:1017B000A354226A144B13400F2BE2D163692269B0
:1017C0001A6122695361FFF763FC104B1A689A4251
:1017D00004D09B699968936899420DD362B621231E
:1017E0000322E35C1340012B0AD0022BD5D1206CDD
:1017F000E16900F035FBD0E70548FFF7E1FBEDE7D5
:10180000E06900F0ADFAC8E7FF00FF00D800002053
:10181000947C0000747C00000000000000000000C8
:1018200038B5114B9C69251C6062A06A2835854239
:1018300006D00368A362FFF74BFDA06AA842F8D167
:101840002223E35C002B08D12123E35C9B0704D116
:10185000226963691A61226953610F20FFF7B8FD9D
:101860000248FFF7ADFB38BDD8000020C07C000067
:1018700010B5041C72B6FFF7F3FB201CFFF7D0FF76
:1018800010BDC04600000000000000000000000085
:1018900010B5041C72B6FFF7E3FB002C02D10B4815
:1018A000FFF78EFB211C0820FFF7BAFDFFF7F0FBC6
:1018B000074B1A689A4207D09B69996893689942C6
:1018C00002D20448FFF77CFB62B610BDB47C000076
:1018D000D8000020947C0000000000000000000000
:1018E00070B50368074D041CAE69002B02D0064892
:1018F000FFF766FB266003207462FFF769FDAB69A2
:10190000586A70BDD8000020647C00000000000010
:1019100070B50468002C0ED02023E35C0E1C051C5F
:10192000032B02D00448FFF74BFB0023201C2B6045
:101930006662FFF7CDFC70BD847C000000000000F3
:1019400008B500290AD0074B42689B6918605A60A5
:10195000136043600420FFF763FD08BD012040428F
:10196000FBE7C046D8000020000000000000000097
:1019700038B50468A0420ED023680D1C036058607F
:101980002023E35C042B02D00348FFF719FB6562B8
:10199000201CFFF79DFC38BDA07C0000000000006B
:1019A00038B572B6FFF75CFB22220A4C2569AB5CA6
:1019B0000133AB54FFF76CFB2368A34207D0A26945
:1019C0009B6892689A4202D20348FFF7F9FA62B61E
:1019D000281C38BDD8000020E47C00000000000076
:1019E000F8B5061C72B6FFF73BFB3469114DAC42EB
:1019F0001ED02227E35DFF2B15D022220133A354F2
:101A0000FFF746FB2B68AB4207D0AA699B68926838
:101A10009A4202D20848FFF7D3FA62B6301CFFF7A9
:101A20009FFE201CF8BD0548FFF7CAFAE35DE4E716
:101A30000024E5E7D8000020E47C0000F07C0000F2
:101A400010B5041CFFF7ACFF03E0FFF7C9FF002847
:101A500002D0C369A342F8D110BDC0460000000007
:101A600010B5041E04D0002324606460A36010BD80
:101A70000148FFF7A5FAF6E70C7D00000000000022
:101A8000F8B53C4B051C9C69FFF792FB002D00D17B
:101A90006BE0A868002863D0A268836820269A4279
:101AA00007D98260835D062B41D0072B2BD0002BFA
:101AB0001ED02B1C03E09A68A1688A4202D31B68DF
:101AC0009D42F8D15A6823606260062014605C6011
:101AD0006562FFF77DFCAB68A34202D02648FFF7A2
:101AE0006FFAA36BAB4202D02348FFF769FAF8BD47
:101AF00001222023C254436802681A6002685360BE
:101B0000FFF7E6FBD5E743680168196001684B60A1
:101B1000416A0B1C02E09E68964202D31B68994200
:101B2000F9D15A680360426010605860C1E74368A9
:101B30000168196001684B60416A0B1C02E09F68F4
:101B4000974202D31B689942F9D15A6803604260F8
:101B5000106058608868A26883689342A1D3A8E7A0
:101B6000A36BAC60EB60A563C1E70348FFF728FAFD
:101B70008FE7C046D8000020287D0000000000004C
:101B800010B5041C72B6FFF76BFA201CFFF778FF44
:101B9000FFF77EFA064B1A689A4207D09B6999684C
:101BA0009368994202D20348FFF70AFA62B610BD61
:101BB000D80000201C7D0000000000000000000094
:101BC000F0B547462D4B80B4061E98469F694BD012
:101BD00072B6FFF745FABB6B002B49D09A68BA4240
:101BE00003D02748FFF7ECF9BB6B9E4202D0244894
:101BF000FFF7E6F9F368BB63FFF7DAFA306886426D
:101C00002FD0BC6BFD6B002C0CD0FFF7D1FA2368F2
:101C10009C4203D09B689D4200D21D1CE468002CAE
:101C2000F3D130680368BD6033605E60836BB06081
:101C3000F3608663FFF74CFBFFF792FCFFF728FA8F
:101C400043461B68434508D0424692699B689268A8
:101C50009A4202D20B48FFF7B3F962B604BC904631
:101C6000F0BD0023B360E9E70548FFF7A9F9AFE746
:101C70000348FFF7A5F9BB6BB0E7C046D8000020CA
:101C8000007D00001C7D000000000000000000003E
:101C9000034A044B1A60044A044B1A607047C0465A
:101CA000280C0020580100200018002054010020BA
:101CB00038B50C1C051CFFF763FA002C13D0631E0B
:101CC0001C4210D10B496B1E0A686042013A1B1975
:101CD0001419094A034012682040121A934206D888
:101CE000C3180B6038BD0548FFF76AF9EAE7002022
:101CF000F8E7C0465801002054010020407D000054
:101D000038B5051C0C1C72B6FFF7AAF9211C281C5B
:101D1000FFF7CEFF041CFFF7BBF9074B1A689A4286
:101D200007D09B6999689368994202D20348FFF7EC
:101D300047F962B6201C38BDD8000020347D000071
:101D400008B50548054B036000238360C36010306D
:101D5000FFF786FE08BDC04660010020011D00009F
:101D6000F0B54746051C80B4002831D043072FD179
:101D7000083D2F686B683E1C0733DB0810376B602B
:101D8000381CFFF7FDFE294B0836341C9846AC4240
:101D900005D863680133DB00E3189D420CD3B442DD
:101DA0000FD0AC420DD32468AC42F8D8636801333D
:101DB000DB00E3189D42F2D24046FFF701F9B4423E
:101DC000EFD12368002B07D09D4205D31C1CDEE712
:101DD0001648FFF7F5F8CBE76A682B602560531CBF
:101DE000DB002968EB188B420BD06268531CDB00C8
:101DF000E3189D4212D0381CFFF7E2FE04BC904667
:101E0000F0BD59681B688C46624401326A606268A2
:101E10002B60531CDB00E3189D42ECD16B689C46A1
:101E20002B686244013262602360E4E7547D000065
:101E300038B5041C0D1CFFF7A3F9002C05D0002DAC
:101E400003D023682B60256038BD0248FFF7B8F83F
:101E5000F7E7C0466C7D00000000000000000000B5
:101E600038B5051C0C1C72B6FFF7FAF8281C211CAB
:101E7000FFF7DEFFFFF70CF9064B1A689A4207D00E
:101E80009B6999689368994202D20348FFF798F8D2
:101E900062B638BDD8000020607D00000000000060
:101EA000EFF30983203383F3098862B67047C04695
:101EB00010B50F300ED072B6EFF30984203C84F3D6
:101EC000098880235B04E361FFF712FB002802D13D
:101ED000024BA36110BD024BA361FBE71C05000090
:101EE00011050000000000000000000000000000DC
:101EF00008B500F0BDFD054800F0E2FE00F058F91D
:101F000001F066FB00F004F808BDC046587F0000F1
:101F100008B500F015FF08BD00000000000000003B
:101F2000F8B5041C0D1C161C1F1C002818D0002915
:101F300016D0012A14D93B1C321D5343EB186361A0
:101F400000236362A362069BA760E362079B25618F
:101F5000E560E761256224606460A2612363F8BDE7
:101F60000148FFF72DF8E6E7787D0000000000004B
:101F700038B5041C0D1CFFF703F92069E3688342A0
:101F800002D008C82B6038BDA368002BF9D0002010
:101F9000F9E7C0460000000000000000000000005B
:101FA00010B5041CFFF7ECF82369E2689A4210D0E0
:101FB000A2680132A260A269944662696344236107
:101FC000934201D3236A2361201C0021FFF7D0FC38
:101FD00010BDA268002AEBD00248FEF7F1FF23698A
:101FE000E6E7C046947D000000000000000000000D
:101FF00038B5041C0D1CFFF7DBF805E0201C291C7C
:10200000FFF79EFC00280DDBA368002BF6D0A36829
:10201000002B08D0E36800201A1D6262A269944672
:102020006344A36238BD0248FEF7CAFFF2E7C04628
:10203000AC7D000000000000000000000000000077
:1020400038B50D1C041CFFF7B3F8002D1CD0A36994
:10205000043B9D4218D8A368002B1BD0E3681D6089
:10206000A268013AA260A269944662696344E3608F
:10207000934201D3236AE36000236362E36A002B87
:1020800001D0201C984738BD0448FEF799FFA3688B
:10209000002BE3D10148FEF793FFDFE7C87D000086
:1020A00070B5041C0E1C151C72B6FEF7D9FF636ACE
:1020B000002B1DD01E70636AA26A013363629342D3
:1020C00010D2FEF7E5FF174B1A689A4207D09B69BA
:1020D00099689368994202D21348FEF771FF62B67D
:1020E000002070BDA369201C191FFFF7A9FFE8E7B6
:1020F000291C201CFFF77CFF051E01D1636AD9E76C
:10210000FEF7C6FF074B1A689A4207D09B69996889
:102110009368994202D20448FEF752FF62B6281C27
:10212000DFE7C046D8000020887D000000000000E6
:1021300010B5041CFFF724F8E268236900209A42D6
:1021400000D010BDA368002BFBD0636A002BF8D031
:10215000043B9B1AF5D01360A368013BA360A369FD
:102160009C4663696244E2609A4201D3236AE36059
:10217000002301206362E4E700000000000000008B
:10218000D62310B5041CC25C0833C25401F070F8A9
:1021900063681B68002B02D0201C01219847032391
:1021A000237010BD000000000000000000000000CF
:1021B00008B500F0EDFF08BD0000000000000000C1
:1021C00001230370002310B54360041C031C00228C
:1021D0004C3388341A60DA6304330021A342F9D106
:1021E0000181418110BDC0460000000000000000D8
:1021F00038B5041C0D1C002829D0002927D072B640
:10220000FEF72EFF2378013B012B02D91248FEF77F
:10221000D7FE231C211C002265600C334C3104C303
:102220008B42FCD1201C00F0CBFF02232370FEF771
:102230002FFF0A4B1A689A4207D09B6999689368E6
:10224000994202D20648FEF7BBFE62B638BD02488C
:10225000FEF7B6FED3E7C046987E0000D800002007
:10226000287E0000000000000000000000000000C8
:10227000F8B5041C0F1C161CFEF782FF002C23D09F
:10228000002E21D02378042B02D01148FEF798FEAF
:10229000BD006519EB68002B02D00D48FEF790FEDB
:1022A000EE607069002803D00021142205F090FB35
:1022B000B069002803D00021142205F089FB391CE5
:1022C000201C00F0E5FFF8BD0148FEF779FED9E7D4
:1022D000147E00000000000000000000000000006C
:1022E000F8B5071CFEF74CFF002F33D03B78042BCA
:1022F00002D01A48FEF764FE01213C1C3E1C00255A
:102300003A897B890A400B403A817B8110344C36F4
:102310002368002B17D072B6FEF7D2FE23685869E7
:10232000002805D002210C304942FFF7F1FA23685A
:102330009869002804D002210C304942FFF7E8FADE
:10234000FEF7D6FE62B620C4B442E1D1381C01F0DB
:1023500067F8F8BD0148FEF733FEC7E7347E00009A
:10236000F0B5474680B4051C0E1C90461F1CFEF7B6
:1023700007FF002D1FD00F2E1DD80123B3406A89FF
:102380009CB2224203D00E48FEF71AFE6A8914431B
:102390004246B31C9B00EB185B686C819B69281C50
:1023A0009A6000221F60311C5A60DA6001F0A0F8C8
:1023B00004BC9046F0BD0248FEF702FEDDE7C046D1
:1023C0004C7E000000000000000000000000000043
:1023D000F0B5474680B4051C0E1C90461F1CFEF746
:1023E000CFFE002D1FD00F2E1DD80123B3402A8908
:1023F0009CB2224203D00E48FEF7E2FD2A89144324
:102400004246B31C9B00EB185B682C815B69281C5F
:102410009A6000221F60311C5A60DA6001F080F877
:1024200004BC9046F0BD0248FEF7CAFDDDE7C04699
:10243000747E0000000000000000000000000000AA
:10244000F8B50223DC21037000230022041C061CC3
:10245000071C0025435202314254013142540C34CE
:10246000038143814C362368002B17D072B6FEF7E8
:1024700027FE23685869002805D002210C30494204
:10248000FFF746FA23689869002804D002210C302F
:102490004942FFF73DFAFEF72BFE62B620C4B44274
:1024A000E1D1C4230022381CFA5400F091FF7B686C
:1024B0001B68002B02D0381C00219847F8BDC0468D
:1024C00038B5E0230278051CC254DB3B0370436837
:1024D0001B68002B01D0042198472C1C4C350C3470
:1024E0002368002B17D072B6FEF7EAFD23685869FF
:1024F000002805D002210C304942FFF709FA236871
:102500009869002804D002210C304942FFF700FAF4
:10251000FEF7EEFD62B60434AC42E1D138BDC046F0
:1025200008B5E023C35C037043681B68002B01D02F
:102530000521984708BDC0460000000000000000CB
:10254000F8B50022C423C254021C041CD43200F08B
:10255000A7FF63689B68002B29D0201C98470028A0
:1025600025D0CC23E1580833E35CDB22DA20A25CDF
:10257000205C120202438A4202D2CC216250111C1A
:102580005BB2002B00DA8DE0002900D078E0052254
:10259000C423E25472B6FEF793FD201C00210022F2
:1025A0000023FFF715FFFEF7A3FD62B6F8BDD427A1
:1025B0006026E35D1E4012D0201C002100F0D0FFF9
:1025C000201C002100F0BCFF63681B68002B02D0B8
:1025D000201C062198470622C423E254E6E7D522B0
:1025E000A55C563A1A402D021543C022920095422E
:1025F00000D101E11CD9C022D200954200D1E0E017
:1026000074D990221201954200D180E0A24A9542ED
:1026100000D1CBE0802212019542CDD1221CC821ED
:10262000DF326250CC22C739A1500432A6509CE759
:10263000022D00D1EAE000D8A9E0802252009542A4
:1026400000D17EE002329542B6D1D622A25C002AA9
:10265000B2D10F21D832A25C114008D052B2201C56
:10266000002A00DA0EE100F08BFFD423E35C0022A5
:10267000C82162500431625004316250002174E775
:102680000422C423E25472B6FEF71AFDC823E258AE
:102690000433E358201C0021FFF762FEFEF728FDFB
:1026A00062B683E7002911D00122C423E25472B636
:1026B000FEF706FDC823E2580433E358201C00212E
:1026C000FFF786FEFEF714FD62B66FE70322C42310
:1026D000E25472B6FEF7F4FC201C00210022002315
:1026E000FFF73EFEFEF704FD62B65FE76B4A9542D8
:1026F00039D0FF32FF32954200D05DE7C8226849E9
:10270000A6500432A6500432A15000212DE7D62550
:10271000DF27625DE15D9142A9D02378042B00D1CF
:102720009BE0002A0AD0DF23E254DB3B237063687E
:102730001B68002B02D0201C02219847D423E35CA5
:1027400095E7D622A25C012A00D035E7DC210220E1
:10275000625A82436252C822A6500432A650043202
:10276000A650002101E7D622A25C002A00D023E770
:102770000F21D832A25C114000D178E752B2201C60
:10278000002A00DA83E000F0DBFEE35D6FE7002D56
:1027900009D1221CC821DC326250CC22C639A1509A
:1027A0000432A550E1E6012D00D005E7C8223D49DD
:1027B000A15002210432A15000210432A150023163
:1027C000D3E6D723D825E15C013BE25C0333E35C2D
:1027D0006068655D1B022B434568201CA8470028E4
:1027E00000D1E9E6C82342680168E2500433E150B1
:1027F0000433E650E35DB8E6D622A25C012A00D09D
:10280000DAE6DC210222605A0243A3E7D8230F2133
:10281000E35C201C5AB21940002A10DB00F010FEC5
:10282000012810D0022800D0C6E6C8231E4A022183
:10283000E2500433E0500433E650E35D95E600F0E7
:1028400017FE0128EED1C823184A0221E2500433B2
:10285000E5500433E650E35D87E672B6FEF730FCE0
:10286000201CFFF73DFDFEF743FC62B60323E6554F
:10287000237063681B68002B02D0201C032198473B
:10288000625D4EE700F08CFED423E35CEFE600F0DF
:1028900067FEE35DEBE6C046020C000002030000A9
:1028A00081210000607E0000647E0000947E0000B4
:1028B000C42310B5C35C041C062B42D82B4A9B00D2
:1028C000D3589F462A48FEF77BFB201C002100F0CE
:1028D00047FE201C002100F033FE63681B68002BBC
:1028E00002D0201C062198470622C423E25410BDC2
:1028F000CC23DA22C0580F33E35CA25C1B021343E3
:10290000834205D9E368198AFDF798FE00291CD097
:102910000322C423E25472B6FEF7D2FB201C00212E
:1029200000220023FFF71CFDFEF7E2FB62B6DEE7A4
:10293000D023C358002B00D098470022C423E25470
:10294000D5E70B48FEF73CFBD1E772B6FEF7B8FBC4
:10295000201C002100220023FFF73AFDFEF7C8FBF0
:1029600062B60222C423E254C1E7C046DC7D000007
:10297000887E000000000000000000000000000051
:10298000C42310B5C35C041C062B37D81D4A9B001A
:10299000D3589F461C48FEF713FB201C002100F073
:1029A000DFFD201C002100F0CBFD63681B68002BBD
:1029B00002D0201C062198470622C423E25410BDF1
:1029C0000522C423C25472B6FEF77AFB201C0021F4
:1029D00000220023FFF7FCFCFEF78AFB62B6EEE75D
:1029E000C3689B695B68002BE9D1D033C358002BC7
:1029F00000D098470022C423E254E0E70248FEF7E3
:102A0000DFFADCE7F87D0000687E000000000000CF
:102A1000031C0A4AC03389019B0099501F230122DD
:102A200003409A40131C054A40099446C022800086
:102A300060445200835003607047C04600E100E0EC
:102A400038B5041C0D1C0B2802D90548FEF7B8FA4E
:102A5000044BA4009C46AD016444656038BDC0468B
:102A6000A47E000018ED00E000000000000000005F
:102A70007047C04600000000000000000000000099
:102A8000882200218020384B520170B59950374977
:102A900080005A5888B002435A501968344A0A4094
:102AA0001A606A46334B694670CB70C270CB70C2F5
:102AB00030CB30C2304B314A9C6C14409C64DC6C8F
:102AC0002240DA648A222E4B1A702E4B863A5A70B4
:102AD0005C781C3222435A7000239A008A58DCB278
:102AE00082423AD00133082BF7D1B8241F21254A5E
:102AF0001470D3780B40D37000231D395371937930
:102B00001942FCD010221F498B791A42FCD10C21AA
:102B10001C4883791B4A0B40082BFAD12021013B2A
:102B200013715133537193791942FCD040211548E8
:102B30008279144B1142FBD00B4A13481349505071
:102B400013491448505000220C211A701A1C937912
:102B50000B400C2BFBD108B070BD3823E4001C40A7
:102B600048331C43C2E7C0460070044038100000E0
:102B7000FFFFF3FF5C7A000000900440FFF8FFFEC7
:102B800000500640004006400000011044100000C4
:102B9000041000000000010100000000000000001F
:102BA00003690120CB4018407047C0460000000078
:102BB00070B5041C0E1C151C1F2924D8062D27D007
:102BC0000122B240636993436361304B9C4227D03A
:102BD0002F4B9C4254D02F4B9C4253D02E4B9C42A7
:102BE00052D02E4B9C4249D02D48FEF7E9F90022E5
:102BF000162D07D82B4BAD005B599F46A023B6007E
:102C0000DB00B35070BD2648FEF7DAF9062DD7D1A8
:102C10000123B3406269134363611C4B9C42D7D1CB
:102C2000214AE5E78023B6005B00B350EAE7812341
:102C3000B6005B00B350E5E70423B600FF33B350A2
:102C4000E0E70023B600B350DCE7E023B600DB008A
:102C5000B350D7E7C023B600DB00B350D2E78023E0
:102C6000B600DB00B350CDE7C023B6009B00B350E5
:102C7000C8E78023B6009B00B350C3E70B4AB7E711
:102C80000B4AB5E70B4AB3E70B4AB1E700F00F4038
:102C900040F00F4080F00F40C0F00F4000F10F40B7
:102CA000207F0000C47E00000090044000D004405B
:102CB00000A0044000B0044000C004400000000038
:102CC000F0B5F82447460E490E4AA4018B5880B44B
:102CD00023438B50A6239B009846071D80443D1C30
:102CE00000243E1FE1B204CD30680134FFF760FFDD
:102CF000202CF7D184374745F1D104BC9046F0BD74
:102D000000700440381000000000000000000000C7
:102D100010B57446FEF704FA72B6FEF7D1F9FEF765
:102D200057F9FEF7E5F962B6FEF712FA201CFFF735
:102D3000BFF810BD0000000000000000000000000F
:102D400008B5064A064B0B205A6000229A600732EB
:102D50001A600821FFF774FE08BDC0467FBB000063
:102D600010E000E000000000000000000000000093
:102D70008B1C9B00C0180223F0B540688900456990
:102D80002C7C23431943038A9A4200D91A1C002A37
:102D900018D000230D4EC900A868C45C70184068A4
:102DA000C45401339342F7D12C7C8823687C1204ED
:102DB00087013B431A4301235840634072506874B3
:102DC0002B74F0BD014EC900EFE7C046000800209B
:102DD000844689008C44F8B56346DF68BD69AB7CE6
:102DE00019437B8A9A4200D91A1C002A25D0002355
:102DF000134EC90074186468A868E45CC4540133B5
:102E00009342F7D17B8A8822EC7C1B04A7013A43CA
:102E10001343735001236340EB746346DB689C6982
:102E20002068002806D0598A01384018FDF780FB39
:102E30002082F8BD01232382FBE7014EC900E2E7AF
:102E4000000800200000000000000000000000005A
:102E5000F0B544465F4656464D468023F0B4C84A16
:102E600083B0D45C7346E4B20193FEF759F963076B
:102E700009D5C4484368DB68002B00D0984704217B
:102E80008023BF4AD154230700D482E0BE4BBD4FFC
:102E90009A469023BA4E9B460CE00D2B00D1FAE0E7
:102EA000012B00D19AE080220823B354B45CE4B231
:102EB00023426ED05B46F35CDBB21C09A21C00927D
:102EC0009200BA185268A10090460422081C1A40C9
:102ED0009210104381464D461B07DB0F58002843D4
:102EE000002B05D143469B69002B00D1C6E09A74A4
:102EF000C300994653464A469A5893061B0F092B1E
:102F0000CBD143465B69002BCDD01A1C002C0BD1D2
:102F1000D422B95C0132BA5C090211431A1CA02305
:102F2000DB00994200D1FEE0494653465B585168A8
:102F30009B019B0D106859185160814200D2C3E07B
:102F400043469B68002BAED00122A2403B899343AD
:102F50003B81009B9B00FB185B689B68002B02D0A9
:102F6000381C211C984772B6FEF7AAF8009B002176
:102F70009D007D196B6858690C30FEF7C9FCFEF79F
:102F8000B7F862B680220823B354B45CE4B223429B
:102F900090D10125254200D0DDE063B2002B00DA9C
:102FA000D5E00223234206D08820754A115CC9B2BD
:102FB000115480215354E30600D59DE0202525427D
:102FC00000D0A5E0FEF7C4F80198FEF771FF03B04A
:102FD0003CBC90469946A246AB46F0BD43469B6931
:102FE000002B00D15FE79201930D994672B6FEF770
:102FF00067F8381C211C4A46FFF7EAFEFEF778F80E
:1030000062B64B46002B00D14DE7434649469B69CB
:103010009A684A449A605A684A445A601A68521A2E
:103020001A601A8A013A92B21A8243465B8A4B4569
:103030005ED94346DB68002B00D134E70122A24071
:103040007B8993437B81009B9B00FB185B68DB685B
:10305000002B02D0381C211C984772B6FEF730F8BE
:10306000009B9D007D196B689B69181C59680C308A
:10307000FEF74EFCFEF73CF862B614E7C300994633
:1030800053464A469B589B061B0F092B00D138E735
:103090000D2B00D007E70223002250460B43DB0034
:1030A000C250032301251943C90042507B89381CB3
:1030B000AB437B8143465B69211C5D7443465B687F
:1030C00098479423F554EEE691688C4663449360E8
:1030D00072B6FDF7F5FF43465A69381C136852680B
:1030E000211C9A1AFFF744FEFEF702F862B6DAE6F0
:1030F000002A00D0D7E69CE722480378042B36D07C
:103100001021802320251E4AD154254200D159E7A1
:1031100084221B4C1B48A35CAB43A354FFF700FA6B
:103120008023E5544EE7D623DE22FB5CBB545F3A96
:1031300013401932B3547B681B68002B02D0381C33
:103140000121984703233B7043465A69ECE68023EC
:103150000B4AD35425E70B48FFF772F98023084A3E
:10316000D554FDF7F5FF0198FEF7A2FE2FE7FFF714
:10317000A7F9842220230249885C03438B54BFE7CC
:1031800000200740940100200008002000000000FB
:1031900008B50548FFF714F880200449044AC00226
:1031A0008B5803438B5008BD9401002000700440ED
:1031B00004100000000000000000000000000000FB
:1031C00038B50378012B00D038BD234B9842FBD192
:1031D000002200202149D300C8500132CB1858608A
:1031E000102AF8D180241E481E4AE4028358234343
:1031F0008350862080231C4C4000225C13432354C0
:103200008625235C184A5BB26D00002BF8DB9C20FE
:103210000B0ADBB213540B0CDBB214301354B4237F
:10322000090ED15480214B33535408315354137435
:10323000515DBF3B0B43535503219423D1540021CF
:103240006C33D1548431505CFF3B034353541820FA
:103250008239FFF7DDFBB7E794010020000800206A
:1032600000700440341000000020074000000000FF
:10327000DE237F22C35C0249134019328B5470470E
:1032800000200740000000000000000000000000D7
:10329000F0B557464E464546E0B482B0102900D9F5
:1032A00083E08B1C9B00C0184668B369002B00D1DB
:1032B00083E000229A74DA74738A414D1B049846A5
:1032C000882340464F0103433E4C7B5123788A00BC
:1032D0003F2B00D96FE02078EF19C0B2431CDBB25E
:1032E0002370394B80019C4601236044786013436E
:1032F0004046C822DB001043585122783F2A5BD851
:103300002078EB18C2B2501C9201C0B26244207007
:103310005A6008237269002A38D0002002241074F1
:1033200050748A001443264F264D9146E200D05136
:10333000A8462D7892463F2D41D845466C462D78BB
:10334000EDB26A1CE271E279AD01944642466446F0
:1033500014701D4A944652466544BC1865604A463E
:1033600003242243D200D051404600783F2800D9A0
:10337000FEE7404645460478BA18E0B2441C800196
:10338000E4B260442C70506004221343032230687E
:103390000240012A03D001200343002A01D0102259
:1033A00013433031094A89008B5402B01CBC90464B
:1033B0009946A246F0BDFEE7FEE70023AAE7FEE736
:1033C00000080020000A00207C02002000200740A6
:1033D000F8B500250E4B94271D7002230D4C0021DB
:1033E000E3550D4B061CC360FFF752FFFF238822F5
:1033F000A354083AA3545E32B554463AA5540C3A45
:10340000A35413327B3BE254833BE355F8BDC046E3
:10341000000A002000200740347F00000000000068
:103420000123002104481A1C303292000133115448
:10343000102BF8D17047C046002007400000000064
:1034400000200F290DD8074B89009C46C0236144FA
:10345000CA5C120705D5C85CBE3B1840421E9041AD
:10346000181A70470020074000000000000000000C
:1034700000200F290DD8074B89009C46C0236144CA
:10348000CA5C520705D5C85CBE3B1840421E90413D
:10349000181A7047002007400000000000000000DC
:1034A000F0B589004018C368104E9F690023BD7CA9
:1034B0000D43ED0074196468E45CD4540133082BA7
:1034C000F8D18822C3685B8A1B041343735101231C
:1034D000BA7C5340C8221943C368C9005B8A1B04E5
:1034E000134373500123FB74F0BDC0460008002055
:1034F000023189004018436810B59C692068002893
:1035000006D0598A01384018FDF712F8208210BD04
:1035100001232382FBE7C0460000000000000000FA
:1035200008B58B1C9B00C3185B685B691A68FFF7C2
:103530001FFC08BD000000000000000000000000AB
:10354000044BC0229C46022389006144885C0343EB
:103550008B5470470020074000000000000000006E
:10356000044BC0229C46022389006144885C0343CB
:103570008B5470470020074000000000000000004E
:10358000044BC0229C460220890061448B5C83432B
:103590008B5470470020074000000000000000002E
:1035A000044BC0229C460220890061448B5C83430B
:1035B0008B5470470020074000000000000000000E
:1035C00008B5FFF75DFA08BD00000000000000002C
:1035D0007047C0460000000000000000000000002E
:1035E000222903D81748890041588F460020704788
:1035F0001548FCE7032AF9D81448D2008018F6E7EA
:10360000042BF3D8124A9B00D3589F46042BEDD8C5
:10361000104A9B00D3589F460F48E8E70F48E6E75B
:103620000F48E4E70F48E2E70F48E0E70F48DEE71E
:103630000F48DCE70F48DAE70F48D8E70F48D6E72E
:103640000F48D4E7EC8100002C830000588500006F
:10365000788200008C8200004C83000024830000EC
:10366000FC850000E08500004483000078850000B0
:10367000E8850000B4820000A8840000E082000019
:10368000B485000000000000000000000000000001
:103690007047C0460000000000000000000000006D
:1036A0007047C0460000000000000000000000005D
:1036B0007047C0460000000000000000000000004D
:1036C0007047C0460000000000000000000000003D
:1036D0007047C0460000000000000000000000002D
:1036E00010B5046B82B02378042B01D002B010BD5A
:1036F00023891B07FAD4064801A9FEF739FC021EEC
:10370000F4D0201C03211023FEF762FEEEE7C04632
:10371000FC0A002000000000000000000000000083
:1037200030B5041C83B072B6FDF7CAFCFDF728FD66
:10373000134DEB68002B02D0281CFDF791FD281CCF
:10374000231C32210F4AFDF75BFDA3690E4D5B6917
:103750001B68002B0FD1281C01A9FEF709FC021ED3
:1037600004D0201C03211023FEF732FEFDF7C0FC1D
:1037700062B603B030BD281CFEF712FCEBE7C04672
:10378000700A002021380000FC0A00200000000020
:1037900070B5041C72B6FDF793FC2378042B22D17C
:1037A000174B1B78002B1ED1164D287800281AD0F5
:1037B00023899B071BD5FA21134B89009C4648435C
:1037C0006044FCF7B5FE8500FDF7DAFC0F4EF368A8
:1037D000002B02D0301CFDF743FD301C291C0C4A85
:1037E000231CFDF70DFDFDF783FC62B670BD201CA8
:1037F0000121084A0823FEF7EBFD2878DBE7C046E5
:1038000031FEFF1FF00A0020E7030000DC0A002061
:1038100091370000300B0020000000000000000085
:1038200030B5051C83B072B6FDF74AFC2B78042B2B
:1038300008D12B891B0705D41A4C201CFEF778FCF5
:10384000002813D1FDF79CFC174CE368002B02D035
:10385000201CFDF705FD201C3221144A2B1CFDF70E
:10386000CFFCFDF745FC62B603B030BD201C01A9BA
:10387000FEF77EFB041E11D0211C01981031231885
:1038800000220F2803D81A7001338B42FBD1281C69
:103890000321221C1023FEF79BFDD3E70448FDF70C
:1038A0008FFBE9E7FC0A0020700A002021380000A5
:1038B000B0840000000000000000000000000000D4
:1038C0007F22D423111C70B5C35C041C194021292C
:1038D00006D0D423E25A664B9A4216D0002070BD1F
:1038E00093432DD0802BF4D15533C35C022B00D1F0
:1038F0008AE0032B53D0012BEBD1D733C35C042BCD
:1039000044D85C4A9B00D3589F46D723D825E15C16
:10391000013BE25C0333E35C6068655D1B022B43A3
:103920004568201CA8470028D8D0C8234268E25028
:1039300002680433E25000220433E2500120CEE753
:10394000D523C35C0A2B64D00B2B0CD0092BC0D120
:10395000CF33C35C002B01D0042BBAD1C823464A15
:10396000E2500122E5E7D823C35A002B0ED1D6330B
:10397000C35C5A1E9341414ADBB21370404A137034
:10398000002B03D13F4D2B78002B4BD10023C822B5
:10399000A3500432A3500432A35001209FE7D82340
:1039A000C35A002B00D094E7C8223449815001212A
:1039B0000432815004328350012090E7C823324AF8
:1039C000C2501022B5E7C823304AC2500522B0E7E2
:1039D000D723C35C012B00D080E7D623C35C022B26
:1039E00040D0032B00D079E7C821294A42501370F8
:1039F000CC2283500022D023C25001206FE7C8237D
:103A0000244AC250102294E7C8231E4AC250012201
:103A10008FE7D7231A4AC35C1A4D12782B70002AFD
:103A2000B2D0B3E772B6FDF74BFBFA211A4B2878F8
:103A30009C46890048436044FCF77AFD8600FDF708
:103A40009FFB164DEB68002B02D0281CFDF708FCED
:103A5000281C311C124A231CFDF7D2FBFDF748FB42
:103A600062B693E70A4A1370C823C250032260E784
:103A700081060000A0820000D80A002000FEFF1F7F
:103A800031FEFF1FF00A0020200A0020F40A002067
:103A9000980A0020300B0020E7030000DC0A002019
:103AA000913700000000000000000000000000004E
:103AB00008B503F03DFF00F09BFC00F079FC08BD69
:103AC00008B503F02DFF08BD000000000000000055
:103AD00010B5041C042929D0052922D0022900D0C0
:103AE00010BD72B6FDF7ECFA201C0121114AFEF759
:103AF000BFFB201C0221104AFEF7BAFB201C032149
:103B00000E4AFEF7B5FB201C04210D4AFEF7B0FB60
:103B1000201C05210B4AFEF7ABFBFDF7E9FA62B664
:103B2000DEE702F025F9FFF7C3FFD9E7FFF7C8FF8B
:103B3000D6E7C04634850000FC83000010850000F5
:103B400054830000BC85000000000000000000005D
:103B500030B5164B164A83B0D358051C5B0306D507
:103B600084221020134952008B5C83438B541248EB
:103B7000FDF78EFE281C1149FEF73AFB8422102324
:103B800000240C495200885C03438B540C4B0D48B5
:103B9000DC600D4B019500930C49F83A0423FEF7C5
:103BA000BFF90B4BDC6003B030BDC04634100000E1
:103BB0000070044000200740DC0500003483000052
:103BC000DC0A0020FC0A0020E1360000200A002068
:103BD000700A00200000000000000000000000004B
:103BE00038B594240423064D0F202A5D13432B552A
:103BF000FDF74EFE04222B5D93432B5538BDC04686
:103C0000002007400000000000000000000000004D
:103C1000014B18787047C046D80A00200000000009
:103C200070B5061C72B6FDF71BFA334C2378042BD3
:103C300010D0FDF72DFA314B1A689A4204D09B69D7
:103C400099689368994201D362B670BD2C48FDF71C
:103C5000B7F9F9E7FDF71CFA284D2B68AB4207D0FE
:103C6000AA699B6892689A4202D22548FDF7A8F992
:103C700062B6244B1B78002B1FD172B6FDF7F0F90A
:103C800023899B072BD40823201C0121321CFEF71B
:103C90009FFBFDF7FDF92B68AB4207D0AA699B6833
:103CA00092689A4202D21648FDF78AF962B610224B
:103CB000311C154803F04CFEC7E772B6FDF7D0F98A
:103CC00023899B0611D41023201C0521321CFEF7EA
:103CD0007FFBFDF7DDF92B68AB42DFD1E6E7236917
:103CE00058690C30FDF7FCFDCDE7236A58690C30AC
:103CF000FDF7F6FDE7E7C04694010020D80000205C
:103D0000C484000031FEFF1F300B002000000000C3
:103D100070B5061C72B6FDF7A3F91B4D2B78042B6A
:103D20000CD0FDF7B5F9194B1A689A4204D09B697B
:103D300099689368994223D362B670BDFDF7A8F9DC
:103D4000124C2368A34207D0A2699B6892689A42EA
:103D500002D20F48FDF734F962B672B6FDF780F96A
:103D60000523281C0221321CFEF732FBFDF790F9D7
:103D70002368A342E0D0A2699B6892689A42DBD292
:103D80000348FDF71DF9D7E794010020D800002073
:103D9000C4840000000000000000000000000000DB
:103DA00010B5041C82B072B6FDF75AF90F480378BB
:103DB000042B0AD1022301AA13706B465C71240AFA
:103DC0009C7104210323FEF703FBFDF761F9084B07
:103DD0001A689A4207D09B6999689368994202D2FF
:103DE0000448FDF7EDF862B602B010BD9401002062
:103DF000D8000020C4840000000000000000000083
:103E000010B5041C82B072B6FDF72AF90F4803788A
:103E1000042B0AD1032301AA13706B465C71240A98
:103E20009C7104210323FEF7D3FAFDF731F9084B07
:103E30001A689A4207D09B6999689368994202D29E
:103E40000448FDF7BDF862B602B010BD9401002031
:103E5000D8000020C4840000000000000000000022
:103E600010B5041C72B6FDF7FBF8164B1B78042B3B
:103E700012D0FDF70DF9144B1A689A4204D09B69D1
:103E800099689368994203D362B6002040B210BD8E
:103E90000E48FDF795F8F7E7FDF7FAF80A4B1A68B0
:103EA0009A4207D09B6999689368994202D2074861
:103EB000FDF786F862B60648211C0122FEF7F0F8ED
:103EC000C0B2E3E794010020D8000020C4840000C1
:103ED000FC0A0020000000000000000000000000BC
:103EE00008B5081CFFF7BCFF08BDC0460000000075
:103EF0007047C04600000000000000000000000005
:103F00007047C046000000000000000000000000F4
:103F100010B501F0FDFEDC23064CE35A9B0700D4EC
:103F200010BD01F00DFF0028FAD0201CFFF758FE4D
:103F3000F6E7C046940100200000000000000000E9
:103F400038B5FDF7D5FFFDF703F8FFF7D1FF1C4C9F
:103F5000201CFFF7FDFD00201A4902F0F9F8237834
:103F6000042B05D03220FDF793FC2378042BF9D1E4
:103F70003220FDF78DFC144802F0FAF800F0C8FA80
:103F8000124800F02DFA03F0A3FC114802F0F0F8FB
:103F9000FFF7B6FF0F4D2378052B0ED1281C02F03A
:103FA000E7F82378052B04D1FFF7B2FF2378052B20
:103FB000FAD001F0C5FB02F0A3FE00F0B1FAEAE787
:103FC00094010020E13E0000048600001CFEFF1F5B
:103FD000188600002C860000000000000000000091
:103FE00038B5184C0321201C0222FEF7E1FD201CED
:103FF00002210222FEF7DCFD134D201C04210222C7
:10400000FEF7D6FD201C07210222FEF7D1FD281C59
:1040100002210222FEF7CCFD281C01210222FEF71C
:10402000C7FD201C094C00210222FEF7C1FD201C07
:1040300011210222FEF7BCFD201C10210222FEF7F6
:10404000B7FD38BDC0F00F4000F00F4040F00F400A
:1040500038B5FFF7C5FF224803210322FEF7A8FD6C
:104060001F4804210322FEF7A3FD1D48002103225F
:10407000FEF79EFD1B4800210322FEF799FD19481B
:1040800003210322FEF794FD164802210322FEF7C6
:104090008FFD154805210322FEF78AFD12480621EF
:1040A0000322FEF785FD0E4801210322FEF780FD65
:1040B000002300220D480E49C252CA520233122B6D
:1040C000FAD102232025FA200A4A054C1178400033
:1040D0000B4313706560FDF7DBFBA56038BDC04680
:1040E00080F00F4040F00F40C0F00F40540B002014
:1040F000680B0020000C0020000000000000000001
:10410000F8B55F464D46564644467C4BF0B49A4659
:104110001F1C7B4B002598467A4B99467A4B9B4651
:10412000082D00D9A9E04A46AB00D3589F46774CEA
:104130001121201C0622FEF73BFD80239B02A36079
:104140002023734E0321F360301CFEF729FD441E2B
:10415000601E84410421301CFEF722FD0138431EFD
:104160009841A4B2400004430021301CFEF718FD22
:104170000138431E98418000044300216348FEF744
:104180000FFD0138431E9841C000044303215F48DE
:10419000FEF706FD0138431E984100010443022149
:1041A0005A48FEF7FDFC0138431E98414001044384
:1041B00005215848FEF7F4FC0138431E9841800160
:1041C000044306215348FEF7EBFC0138431E984197
:1041D000C00104430121301CFEF7E2FC0138431EFC
:1041E00098413B8800020443A3420BD043461B780E
:1041F0003C80002B03D05B461B78DB0764D405238F
:10420000424613700135EDB2FFF7EAFE0237092D81
:1042100086D143461B78002B0DD04246013BDBB2D2
:104220001370002B65D100233B495246D25ACA5223
:104230000233122BF9D101203CBC90469946A2468C
:10424000AB46F8BD334C0021201C0622FEF7B0FC23
:104250000123A36074E72F4C0421201C0622FEF7E3
:10426000A7FC1023A3606BE72A4C201C0221062226
:10427000FEF79EFC0423A36062E7264C0321201C6A
:104280000622FEF795FC0823A36059E7234CECE7D0
:10429000204C0721201C0622FEF78AFC8023A36005
:1042A0004EE71E4C0121201C0622FEF781FC022352
:1042B000A36045E7154C1021201C0622FEF778FC70
:1042C00080235B02A3603BE7154801F051FF5B468A
:1042D0001B78DB0793D543461248197801F048FF55
:1042E0005B461B78DB0700D489E70F4801F040FFED
:1042F00085E70120FDF7CCFA9DE7C046680B00205A
:1043000030FEFF1FD8860000000C002040F00F4058
:1043100080F00F40C0F00F40540B002000F00F4021
:10432000FC86000008870000F091000000000000FB
:10433000014B4000185A7047540B00200000000049
:10434000F8B54F4646461248C0B401F011FF114B74
:1043500000249946104B114F9846114E114D211CC7
:10436000484601F005FF404601F002FF6300F85A9D
:1043700001F06EFC011C301C01F0FAFE0134281C17
:1043800001F0F6FE092CEAD10CBC90469946F8BD26
:10439000108700000887000028920000540B0020BE
:1043A00028870000F09100000000000000000000DD
:1043B00010B5830705D4074805210222FEF7F8FB54
:1043C00010BD044C0521201C0622FEF7F1FB202322
:1043D0006360F5E780F00F4000000000000000007F
:1043E000014B18607047C046800B002000000000A1
:1043F00008B5044B1B68002B02D01B68984708BD0A
:104400000020FCE7800B00200000000000000000FE
:10441000F8B5194B1B68002B21D05B68041C98472A
:10442000164D2B785A071AD5DB07DB0FDBB2002BB2
:104430001AD1261C124F103602E00134B4420CD0BF
:10444000002BFAD02178381C01F092FE2B78013431
:10445000DB07DB0FDBB2B442F2D1002B00D1F8BD99
:10446000084801F085FEFAE7074801F081FE2B7845
:10447000DB07DB0FDBB2DCE7800B0020000C002049
:1044800044870000F0910000308700000000000029
:1044900008B5034B1B68002B01D09B68984708BDEB
:1044A000800B002000000000000000000000000061
:1044B00008B5064B1A88824206D01880044B1B6848
:1044C000002B01D0DB68984708BDC0467C0B00205C
:1044D000800B002000000000000000000000000031
:1044E00008B5064B1A88824206D01880044B1B6818
:1044F000002B01D01B69984708BDC0467A0B0020ED
:10450000800B002000000000000000000000000000
:1045100008B501F045FEFFF79BFD01F009FF08BD5E
:10452000F0B556465F464D464446F0B483B0FFF7BB
:10453000E7FD3D4B00259A463C4B01269B46EBB2DE
:10454000181C9946FFF7F4FE6B0098465346424606
:104550009C5A071C4440A4B2002C0CD05B461B782C
:104560009B071CD40023221C1A41D9B2164219D130
:104570000133092BF7D10135092DE0D16A46FF231C
:10458000137053700023937001F012FE012318433F
:104590006B4698800199009800F05AF821E0FFF7E7
:1045A000CFFEDFE701249C406A46274011707B1E46
:1045B0009F4149469770517001F0FAFD012318435D
:1045C0006B4698800199009800F042F80199009894
:1045D00001F076FB4246534641469B5A52466340A1
:1045E000535201F065FB02F0FBFBFFF701FF104C9B
:1045F000237883420AD0FFF7FBFE0C4B011C1B788B
:1046000020705A0709D4081C01F072FB03B03CBCAF
:1046100090469946A246AB46F0BDDB07F3D5054868
:1046200001F0A6FD2178EEE7840B0020000C0020AD
:10463000960B00204C8700000000000000000000E6
:1046400008B5FFF7B5FE08BD00000000000000003F
:10465000F0B5041C031C87B0240A02AA8DB2009096
:104660000191C6B20293E4B2181C9180002D08D0CB
:104670001670547012880A4B9A4202D0019901F0C8
:104680001FFB002205926A4616705470009A04AB14
:1046900004929D800098059900F042FE07B0F0BD9D
:1046A000FFFF00000000000000000000000000000C
:1046B00010B5002820D0041E822C6AD083284FD049
:1046C000842800D174E0031FDBB2A02B57D9031C50
:1046D0002033DBB2072B00D879E0031C5B33DBB25D
:1046E000022B0AD8A52800D17DE0A63844426041BB
:1046F0008323181AFFF7DCFE10BD031C5833DBB20E
:10470000142BF9D8A8286CD0A9286ED0AA286ED06E
:10471000AB286ED0AC286ED0AD286ED0AE286ED04F
:10472000AF286ED0B1286ED0B0286ED0B2286ED02F
:10473000B3286FD0B42870D0B52871D0B62872D005
:10474000B72875D0B82870D0B92875D0BA2871D0DC
:10475000BB2875D0BC2871D00020FFF7C1FECBE785
:10476000FFF746FEC307C7D4532001F019F800F045
:10477000E7FF532001F064F800F0E2FFBCE702F02D
:104780003FFF0028B8D1201C01F00AF800F0D8FF44
:10479000B2E7FFF72DFE8307AED4392001F000F811
:1047A00000F0CEFF392001F04BF800F0C9FFA3E77D
:1047B000FFF71EFE43079FD4472000F0F1FF00F0F3
:1047C000BFFF472001F03CF800F0BAFF94E7072054
:1047D00001230440A340D8B201F08AF800F0B0FFF2
:1047E0008AE7E220B9E7812084E7E920B5E7EA20FB
:1047F000B3E7B520B1E7B620AFE7B320ADE7B4200B
:10480000ABE7B720A9E7CC20A7E7CD20A5E7842018
:10481000FF30A2E7C52040009FE7C92040009CE789
:10482000CA20400099E7074897E78920800094E76D
:10483000054892E7054890E705488EE705488CE76C
:1048400005488AE72102000023020000260200003A
:10485000250200002A0200002702000000000000DC
:1048600008B500281AD082282CD0832817D0842895
:1048700046D0031FDBB2A02B33D9031C2033DBB29D
:10488000072B33D9031C5B33DBB2022B16D958300C
:10489000C0B2142802D80020FFF722FE08BDFFF79F
:1048A000A7FDC307FAD5532000F07AFF00F048FFB8
:1048B000532000F0C5FF00F043FFEFE70020FFF7B3
:1048C000F7FDEBE7FFF794FD8307E7D5392000F00C
:1048D00067FF00F035FF392000F0B2FF00F030FF35
:1048E000DCE700F0ADFF00F02BFFD7E7072318400F
:1048F000063B8340D8B201F003F800F021FFCDE77A
:10490000FFF776FD4307C9D5472000F049FF00F0C7
:1049100017FF472000F094FF00F012FFBEE7C046EB
:10492000F0B54746041C80B484B0211C06226846BA
:1049300003F00EF8A37921781D09A3886278A7787F
:10494000002B3BD002AB19705A701888B64B9842B6
:1049500034D06B465A701970009800F0C9FE061CDE
:1049600000F0BEFE00F0F4FD3204130F0F2B25D82B
:10497000AE499B00CB589F46002F00D111E1F305B3
:10498000DB0F002B1AD033065B0F9B003407DBB222
:10499000240F9C400020F20602D50F309840C043FF
:1049A0003605B60F022E00D156E1032E00D12DE1BF
:1049B0002043012E00D12CE100F072FE04B004BCB3
:1049C0009046F0BD3005020FF1B2201C01F090F8C6
:1049D00000F02EFDF2E70F23120E34059A43240F48
:1049E000002A01D02401E4B2002F00D1CDE0002C38
:1049F00000D0D9E0F0B2FFF75BFEDFE70F23120E25
:104A00009A4333051B0F202A01D01B01DBB2F0B201
:104A10009846002800D1ADE0012800D096E0002F94
:104A200000D1EAE0052DC9D800F05AFF4346034201
:104A300000D1A5E0404600F063FF00F081FEBDE735
:104A400033059B0F7BD0012BB8D1002F00D1B1E0F3
:104A5000B005800DFFF744FDB0E7F0B2002F69D03C
:104A600002F00EF802F04CF9A8E79201920F00D084
:104A700082E7002FA2D133065B0F9B003407DBB225
:104A8000240F9C400020F20602D50F309840C0430E
:104A90003605B60F022E00D1E2E0032E00D1AFE0C2
:104AA0002043012E00D1AEE000F07AFD86E7F4B29B
:104AB000231C2033DBB2132B00D97FE05C4A9B0020
:104AC000D3589F463005020FF1B2201C01F018F8B0
:104AD00074E7002F06D0F004C00E00F0B1FD6DE7C2
:104AE000002FF8D0F004C00E00F09AFD66E7002F0A
:104AF00000D1AAE0042D00D960E7F004C00E00F058
:104B0000AFFD5BE7F004C00E002F00D192E000F093
:104B100087FD0F20204000D150E700F0E9FE00F0B3
:104B20000FFE4BE7002F00D193E0F004C00E00F021
:104B300067FD43E702F02CF802F0E2F83EE7002FB1
:104B400050D0B005800DFFF7B3FC37E7002F4DD0F4
:104B5000002D15D0A379DA0735D50F221340A371A4
:104B60004346002B00D129E7404600F0C1FE00F08B
:104B7000E7FD23E7002F29D0002D01D0012D73D0B0
:104B80004346002B00D119E7EEE7F0B2FFF768FECD
:104B9000002C00D112E7201C00F0D2FE00F0D0FD66
:104BA0000CE7B305DB0FECE6201C00F0C1FE00F0C3
:104BB000C7FD1FE70020FFF793FCFFE6002F2BD077
:104BC000002D8FD0201CFFF773FDF7E6002D02D0DB
:104BD000012D00D1F2E600F0CBFE4346002B00D1C0
:104BE000ECE627E70020FFF763FCE7E6002D17D18E
:104BF0004346002B00D1E1E61CE7042DF8D9DDE6A1
:104C000000F0CEFC201C00F0BBFCD7E600F048FD15
:104C1000201C00F035FDD1E6002D00D15BE7201C03
:104C2000FFF71EFECAE6C046FFFF000058870000DF
:104C30009887000000F004FD0F20204000D1BDE661
:104C400000F05EFE00F07CFDB8E6052D00D9B5E66B
:104C500053E700F0C5FCB1E6204300F031FDADE6BE
:104C6000204300F0ADFCA9E6181C00F079FEA5E693
:104C700008B500F06DFE00F023FE00F061FD02F0CB
:104C80005FF902F03DF80020FFF712FC0020FFF76B
:104C900027FC08BD0000000000000000000000002C
:104CA00008B500F03DFEFFF7E3FF08BD000000007F
:104CB00010B582B001AB1880019800F019FD030413
:104CC0001B0F023B00220D2B0FD801210C1C9C4016
:104CD000231C9024A40123420AD108490B4204D08A
:104CE000C3B2DF2B08D9F02B06D0101C02B010BDC8
:104CF000C00A021C0A40F8E70122F6E7030300009D
:104D000082B002B07047C046000000000000000002
:104D100082B002B07047C0460000000000000000F2
:104D2000F8B50A4B0A4E1C783378A3420CD00727FB
:104D3000084DE300E858EB185968FFF7E9FF3378AE
:104D400001343C40A342F4D1F8BDC046E00B002042
:104D5000E10B0020980B0020000000000000000084
:104D6000F0B55F4656464D464446F0B4344885B0EB
:104D700083791B0906D005B03CBC90469946A246F3
:104D8000AB46F0BD8378002BF5D02E4B2E4D1B7813
:104D90002A789A42EFD02D4A072694462C4A90460C
:104DA000C722914604E02A78013333409A42E2D088
:104DB000026802A9029282888A8004784178002AD7
:104DC000F1D002AF3C7079703F886745EBD0DF00CF
:104DD000BA46C244019757467F788F42E3D1414695
:104DE000019FC95DA142DED1514689780029DAD1FF
:104DF0005446A488A2421BD96746BA1A4F461419D2
:104E0000E20FA7425141C9B20029CCD00F21102294
:104E100083790B4013438371019B43441F1C9B798F
:104E20000B401A43BA71FFF77BFDFFF779FFA2E74A
:104E30004F46A21AD40F97426141C9B2E4E7C04677
:104E4000D80B0020E00B0020E10B0020FFFF00004A
:104E5000980B00200000000000000000000000008F
:104E6000F0B544465F4656464D46F0B4051C99B031
:104E7000291C062204A802F06BFD2B78C64C9C4628
:104E80006B780393AB789846AB880293216806ABA6
:104E90000691A7888A469F80627820780192002F29
:104EA00059D06A46127918705A701E88BB4B9E42C0
:104EB00002D0A678002E69D1524610926A4610ABF5
:104EC0009F80127918705A701E88B44B9E4242D04F
:104ED000A678002E3FD1029A974200D9F3E0D71B63
:104EE000C722FB0FBA425E41F6B2002E00D15CE150
:104EF0004646002E32D0226812AB12926A46A7882C
:104F000018709F8012795A701988A44B99420AD060
:104F1000614604AA11706946097B23885170118883
:104F2000994200D10FE1624604AB1A706A46127BC7
:104F30005A700498FFF7BCFE002800D1FBE0291C42
:104F40000822201C02F004FDFFF70AFF03CCFFF744
:104F5000DFFE012606E04346002B0BD1281CFFF79D
:104F6000DFFC0126301C19B03CBC90469946A24695
:104F7000AB46F0BD6A466146127B04AB19705A70AD
:104F80000498FFF795FE0028E8D0D8E7029A9742E8
:104F90004CD9029ADB1B91464B44DA0F9346002210
:104FA0009146C72749465A469F424A41D3B299463D
:104FB0004B46A779002B49D00F239B463B1C5A46F2
:104FC000934300D089E0226808AB089292466A4673
:104FD000A68818709E8012795A7019886F4B994272
:104FE0000AD0614604AA11706946097B2388517072
:104FF0001188994200D16CE1029B4646002B00D1FA
:10500000CEE062460AAB1A706A46127B5A70198863
:10501000624B994200D1C3E04346002B00D1DAE055
:105020000123A27900261343A3719BE7D71BC72254
:10503000FB0F9946934600234A465946B9425341CD
:10504000DBB299464B46A779002BB5D10F233A1C0A
:105050009A4300D10AE122680EAB0E92A288187022
:105060009A806A4612795A7019884C4B99420AD034
:10507000614604AA11706946097B23885170118822
:10508000994200D17BE0624604AB1A706A46127BFB
:105090005A700498FFF70CFE002800D15EE74346E3
:1050A000002B00D15AE7A3791F2B00D847E716A899
:1050B00022880280002282706A461289837182806F
:1050C000FFF72EFC3BE7029ADB1B9146C7274B44B8
:1050D000DA0F9F425641F6B207E722680CAB0C92FA
:1050E0006A46A68818709E8012795A7019882B4BD0
:1050F00099420AD0614604AA11706946097B238847
:1051000051701188994200D1CBE0624604AB1A700D
:105110006A46127B5A700498FFF7CAFD002800D136
:105120001CE74346002B00D118E7A3791F2B00D8BA
:1051300005E714A8BCE70123A279281C1343A37137
:10514000FFF7EEFB0EE7A379DA0700D5BBE01A09FB
:1051500000D1B8E0AB710F2A05D00F210132120146
:105160000B401343AB71281CFFF7DAFB291C201CF2
:10517000082202F0EDFB03CCFFF7CAFDF2E643463E
:10518000002B00D07FE7AF71281CFFF7C9FB434617
:1051900023606360E6E6C046D80B0020FFFF0000F6
:1051A0004346002B00D1DDE63AE7624604AB1A70B5
:1051B0006A46127B5A7042469A706A4612899A80F1
:1051C00004980599FFF79CFD002000212660666089
:1051D000FFF79EFDC6E64D4B4D491B780A78904679
:1051E000934221D007226146281C9246B446454688
:1051F000484F039A80460E1C04E0514601330B4091
:10520000AB420CD0D900781844789442F5D1795C3F
:10521000B142F2D181780029EFD06646A2E6331C74
:10522000454666469C460392624604AB1A706A463F
:10523000127B5A70049800F05BFAC2B20004030FAC
:10524000012B4EDD032B0CDC0F23000E034203D099
:10525000A979994300D185E62032D2B2072A00D835
:1052600080E6281CFFF75CFB4E467BE6624604ABFB
:105270001A706A46127B00265A7042469A706A4635
:1052800012899A8005990498FFF73AFD201CFFF7D0
:1052900047FB4B460020002123606360FFF738FD89
:1052A00060E64346002B00D02FE7281CAF71FFF7C4
:1052B00037FB201C291C082202F04AFB03CCFFF715
:1052C00027FD4E464EE6201C291C082202F040FB1A
:1052D00048E64646002E0AD0029B002B00D19FE6EE
:1052E0008FE60001000FB7D0002AB5D13AE65A4642
:1052F00010233A401343A37150466168FFF708FD3D
:10530000201CFFF70DFBA379AB712BE6E00B00200F
:10531000E10B0020980B00200000000000000000BE
:10532000F0B5474680B488B0009068460191FFF719
:1053300097FD6C46051E38D0009802AB0290A288FB
:105340009A80A28825786178002A20D1324E334C89
:1053500033782078984216D0314D07270DE0237816
:10536000DB00E858EB185968FFF7D2FC2078337857
:10537000013038402070834205D0C0002818FFF764
:105380006FFD0028EBD108B004BC9046F0BD1D7045
:1053900059701A88234B9A42D8D00199FFF7B8FC6C
:1053A0001D4E1E4C33782078D4E706AF3B1C6A466E
:1053B00003CA03C323786678A4883B707E70BC80E0
:1053C00004A8391C0622984602F0C2FA002CBDD06F
:1053D0006B4642465E741A741A8A124B9A42B5D0D2
:1053E00007210D4E0D4C33785A1C0A4021788A4211
:1053F0000AD00B4DDB00ED180ACF0AC53270FFF75B
:105400008FFC33782078A5E7FFF74AFC064B357010
:1054100025701D605D60B6E7E10B0020E00B002009
:10542000980B0020FFFF0000D80B002000000000B8
:10543000F0B557464E464546E0B4071E43D07F239D
:105440009846783B00260025994638787C1C7528BC
:1054500020D0752821D873283AD8042862D2012890
:105460004FD002282FD17878BC1C031C2033DBB22C
:10547000072B60D9FFF7F4F9271C2C1EE5D0013C5F
:105480000120E4B2FCF704FA002CF8D138787C1C37
:105490007528DED17D780237EFE778282BD00AD83F
:1054A000762823D077280ED1301C00F031FA271C43
:1054B00000F046F9E1E7031C7C33DBB26F2B02D826
:1054C00043461840D6E71CBC90469946A246F0BD1C
:1054D0007C78BB1C9A46002C06D0013C0120E4B22B
:1054E000FCF7D6F9002CF8D15746C6E700F0F8F9DA
:1054F000271C061CC1E700F013FA271C00F020F956
:10550000BBE77B78BC1C1A1C2032D2B2072A0DD80C
:105510004A4613409840C0B200F00AFA271C00F037
:105520000FF9AAE7FFF7C4F8271CA6E7181CFFF736
:10553000BFF8271CA1E74B46184001238340D8B28F
:1055400000F0FEF9271C00F0FBF896E700000000D1
:105550007047C0460000000000000000000000008E
:1055600008B5034B186000F0B3FBFFF781FB08BDE3
:10557000E80B002000000000000000000000000018
:1055800008B5044B1A681043186000F0A1FBFFF740
:105590006FFB08BDE80B00200000000000000000C9
:1055A00008B5044B1A681040186000F091FBFFF733
:1055B0005FFB08BDE80B00200000000000000000B9
:1055C00008B5044B1A685040186000F081FBFFF7E3
:1055D0004FFB08BDE80B00200000000000000000A9
:1055E000002208B5034B00201A6000F079FBFFF79A
:1055F0003FFB08BDE40B002000000000000000009D
:1056000008B501238340181C034B186000F068FBA9
:10561000FFF72EFB08BDC046E40B00200000000091
:1056200008B501238340181C044B1A681043186006
:1056300000F056FBFFF71CFB08BDC046E40B002042
:1056400008B501238340181C044B1A688243101CC0
:105650001A6000F045FBFFF70BFB08BDE40B0020D0
:1056600008B501238340181C044B1A685040186089
:1056700000F036FBFFF7FCFA08BDC046E40B002043
:1056800008B5044B1A681043186000F029FBFFF7B7
:10569000EFFA08BDE40B002000000000000000004D
:1056A00008B5044B1A681040186000F019FBFFF7AA
:1056B000DFFA08BDE40B002000000000000000003D
:1056C00008B5044B1A685040186000F009FBFFF75A
:1056D000CFFA08BDE40B002000000000000000002D
:1056E0007047C046000000000000000000000000FD
:1056F000F0B583B00E4B01AF38801D680D4B1F24F1
:105700001B6801261D4301E0013C0CD32B1CE34028
:105710001E42F9D0E0B2396800F01AFA80B20128CE
:10572000F2D003B0F0BD0199002000F011FAF8E7C3
:10573000E80B0020E40B0020000000000000000047
:1057400038B5104B104D1868104B1A78104B1B7859
:1057500013432A780370002A11D0041C134300223B
:1057600003701034431C1978002901D00132D2B2E1
:105770000133A342F7D1002A01D000232B70FEF79A
:1057800047FE38BD34FEFF1FED0B0020EC0B002060
:10579000EE0B0020000000000000000000000000F0
:1057A000F8B51F4B011C1B78002B03D01D4B1B7839
:1057B000002B1DD11C4BFF251E68371C331C0E37D8
:1057C00002E00133BB420DD098789A1BD2B28142DD
:1057D0000DD06CB20134F4D10028F2D10133151C84
:1057E000BB42F1D16DB26B1C01D07519A970F8BD27
:1057F000C3080E2B07D90D4B1B78DB07F7D50C48D8
:1058000000F0B6FCF3E7084A106807221140063A98
:105810008A40111CC3185A7811435970E7E7C046F3
:1058200000FEFF1F31FEFF1F34FEFF1F000C002093
:10583000E8870000000000000000000000000000F9
:1058400010B5184B1B78002B03D0174B1B78002B7F
:1058500010D1164B00211C68A31C103402E0013348
:10586000A34206D01A788242F9D119700133A342BB
:10587000F8D110BDC3080E2B08D90D4B1B78DB07E0
:10588000F7D5011C0B4800F073FCF2E7074A1168DA
:1058900007221040063A8240101CCB185A788243E7
:1058A0005A70E6E700FEFF1F31FEFF1F34FEFF1FA8
:1058B000000C00200888000000000000000000002C
:1058C0000021044B1A68531C1032197001339342A3
:1058D000FBD1704734FEFF1F0000000000000000F5
:1058E000014B18787047C046EE0B00200000000006
:1058F000024A1378184310707047C046EE0B002020
:10590000024A1378834313707047C046EE0B0020A1
:10591000014B18707047C046EE0B002000000000DD
:105920000022014B1A707047EE0B002000000000AF
:10593000024A1378184310707047C046EC0B0020E1
:10594000024A1378834313707047C046EC0B002063
:105950000022014B1A707047EC0B00200000000081
:10596000014B18707047C046ED0B0020000000008E
:105970000022014B1A707047ED0B00200000000060
:1059800008B5031EBC2B09D8A82818D2A4284BD8C8
:10599000042847D20120012B0FD108BDE7283BD8AE
:1059A000E0283FD2BF2808D1FFF77AF93220FBF771
:1059B0006FFF00F065FC0020EFE70020EDE7A8286E
:1059C0003ED0A9283AD0AA283ED0AB2834D0AC2863
:1059D0003CD0AD283CD0AE283CD0AF283CD0B1283C
:1059E0003CD0B0283CD0B2283CD0B3283CD0B4281E
:1059F0003CD0B5283CD0B6283CD0B7283CD0B828FD
:105A00003ED0B9283AD0BA2840D0BB283CD0BC28D8
:105A100038D08820C001C0E7F028CED3A020C00134
:105A20001843BAE7181CB8E7A5280BD0A63B584284
:105A300043411748C01AB0E71648AEE71648ACE72E
:105A40001648AAE71648A8E71648A6E71648A4E7A6
:105A50001648A2E71648A0E716489EE716489CE7B6
:105A600016489AE7164898E7164896E7164894E7C6
:105A7000164892E7164890E716488EE716488CE7D6
:105A800016488AE7164888E7164886E7164884E7E6
:105A900083400000B5440000E9440000E2440000F7
:105AA00081400000EA440000B6440000B344000016
:105AB000B4440000B7440000CC440000CD440000D2
:105AC000834500008A45000092450000944500008F
:105AD0002146000023460000254600002446000021
:105AE0002A4600002746000026460000000000006D
:105AF00000207047000000000000000000000000CF
:105B00007047C046000000000000000000000000D8
:105B10008BB21B0ADA00D218C3001818C300C018D1
:105B2000034B1018C9B21818405C82B002B070471D
:105B300034860000000000000000000000000000AB
:105B4000024BC0384000C05A7047C0463086000043
:105B500000B583B001AB19800199FFF7D9FFDF28A9
:105B60000FD8C02845D231285ED01ED8292839D078
:105B70002A2849D1334B2A201B785B0613D53120C4
:105B800011E0E32857D01DD8E02846D0E2283BD1C9
:105B90002C4B1B785A0752D5DB06DB0F5A42534178
:105BA000E3205B42184003B000BD392824D082288E
:105BB00022D0352828D1234B35201B789B06F2D5DF
:105BC0002920F0E7E62822D0E7281DD11D4B1B78BD
:105BD0001A0720D4DB06DB0F5A425341E7205B4211
:105BE0001840E0E7174B29201B789B06DBD53520B2
:105BF000D9E7FFF7A5FFD6E7124B1B78DA0701D4E8
:105C00009B0701D5E020CEE7FFF7BAFECBE70D4BAF
:105C10001B781A07DED4E620C5E70A4BE0201B7884
:105C2000DB07C0D53920BEE7064B31201B785B0669
:105C3000B9D52A20B7E7034B1B785A07ACD5E22029
:105C4000B1E7C0460C0C002000000000000000007E
:105C5000C3B270B5000A1D011B0902012B430009E4
:105C6000DDB210433321C2B22C1C131C8C430D40F7
:105C7000AD008B43A41011402C4389009B10552686
:105C8000251C0B43191CB5436D10B1433340281C30
:105C900049105A000B1C3440640020431343000297
:105CA000184370BD0000000000000000000000006C
:105CB0007047C04600000000000000000000000027
:105CC00082B002B07047C046000000000000000033
:105CD0007047C04600000000000000000000000007
:105CE0007047C046000000000000000000000000F7
:105CF00008B5FEF7A5FC08BD00000000000000008C
:105D00007047C046000000000000000000000000D6
:105D100008B51120FBF7BCFD08BDC046000000001F
:105D20007047C046000000000000000000000000B6
:105D30007047C046000000000000000000000000A6
:105D400010B5FFF7EDFF0024FEF7DAF9FFF7F0FFDB
:105D5000201CFEF7EDFA002804D10134E4B2092C2E
:105D6000F6D110BD0120FCE700000000000000009B
:105D700008B5FFF7D5FDFFF7EBFDFFF7A1FD01F03B
:105D8000DFF80020FEF794FB0020FEF7A9FB08BD1A
:105D9000F0B54E46574645469146E0B40124051CF1
:105DA0000E1C1F1C884208D37443281C211CFAF7C0
:105DB000BFFBB042F8D2002C29D000239846211C0A
:105DC000281CFAF7B5FB211C8246281CFAF736FC82
:105DD000201C0D1C311CFAF7ABFB4346041C002BA6
:105DE00002D15346002B1ADD52467B1C3020092A73
:105DF00004DD4A460730002A00D1203001229446B3
:105E000050443870E044002C02D01F1CD7E73B1CE4
:105E100000221A701CBC90469946A246F0BD00288C
:105E200002D03B1C1F1CCAE7504630307B1C387028
:105E3000EEE7C04600000000000000000000000087
:105E4000F0B54E46574645469146E0B40124051C40
:105E50000E1C1F1C884208D37443281C211CFAF70F
:105E600067FBB042F8D2002C29D000239846211CB1
:105E7000281CFAF75DFB211C8246281CFAF7DEFB82
:105E8000201C0D1C311CFAF753FB4346041C002B4D
:105E900002D15346002B1ADD52467B1C3020092AC2
:105EA00004DD4A460730002A00D120300122944602
:105EB00050443870E044002C02D01F1CD7E73B1C34
:105EC00000221A701CBC90469946A246F0BD0028DC
:105ED00002D03B1C1F1CCAE7504630307B1C387078
:105EE000EEE7C046000000000000000000000000D7
:105EF000F0B54746061C80B430240F1C002B00D19F
:105F0000103C069B01339846069B1978002923D044
:105F1000002A16DD434602E00133002A11D018782A
:105F2000013A0028F8D1551E002A0AD0301C211C45
:105F3000013DB8476B1C002BF8DC069B1978002943
:105F400007D04446301C0134B847631E1978002935
:105F5000F8D104BC9046F0BD551E002AE6DCF8E7F7
:105F6000F0B55F464D4644465646F0B41F1C2D23FF
:105F700081468846151C9B4689B02978002907D0A0
:105F800025290CD001354846C04729780029F7D18A
:105F900009B03CBC90469946A246AB46F0BD6B7832
:105FA000302B53D000229246AE1C1A1C303AD1B28C
:105FB000002409291CD96C2B35D0632B67D04AD912
:105FC000732B51D06AD9752B77D1351C3B1D0393A8
:105FD00038680A21002205ABFFF732FF039F05ABAB
:105FE000009348464146221C5346FFF781FFC4E711
:105FF000311C0AE00A320A2ADDDCA3001C190B78E6
:10600000640014191A1C0131303AD0B20E1C092850
:10601000F3D91A1C613A052AECD91A1C413A052A0F
:10602000E8D96C2BC9D13378751C632B2ED052D98B
:10603000732B18D065D9752B55D138683E1D0A21B0
:10604000002205ABFFF7A4FE371CC8E70122EE1CB7
:10605000AB789246A9E7252B13D0582B2FD0002BD5
:1060600096D0351C89E72E1C3B683D1D00934846A1
:106070004146221C00232F1CFFF73AFF351C7CE70A
:106080002E1C48462521C047351C76E72E1C397842
:106090003C1D4846C047271C351C6EE7642BE0D1E9
:1060A00038683B1D0393002842DB05AB0A21002220
:1060B000FFF7C6FE351C039F91E7782BD1D1583BE3
:1060C0003D1D38685A425A41102105AB2F1CFFF77D
:1060D000B7FE351C83E7252BD2D0582B06D0002BDA
:1060E00000D155E749E7782B00D046E7583B3868A0
:1060F0005A425A413E1D102105ABFFF749FE371C9D
:106100006DE7642B00D038E738683E1D002806DBB9
:1061100005AB0A210022FFF73BFE371C5FE75A461A
:1061200002AB1A7302AA0D23944640426344F0E77F
:106130005A4602AB1A7302AA0D23944640426344A6
:10614000B4E7C046000000000000000000000000AE
:10615000024B1960024B18607047C046040C0020C7
:10616000080C0020000000000000000000000000FB
:106170000FB400B5064983B004AB0868054904CBE9
:1061800009680193FFF7ECFE03B008BC04B01847A0
:10619000080C0020040C002000000000000000009B
:1061A0007047C04600000000000000000000000032
:1061B00038B572B6FAF754FF0C4DAC6AFAF768FFBF
:1061C0002B68AB4207D0AA699B6892689A4202D2B8
:1061D0000748FAF7F5FE62B6FA21013489004C430C
:1061E000601EFAF7A5F980B238BDC046D80000207D
:1061F00028880000000000000000000000000000EF
:1062000038B572B6FAF72CFF0B4DAC6AFAF740FFBF
:106210002B68AB4207D0AA699B6892689A4202D267
:106220000648FAF7CDFE62B6FA21013489004C43E4
:10623000601EFAF77DF938BDD800002028880000DC
:1062400038B5FA25094BAD009C6A094B68439C465A
:10625000291C6044FAF76CF90134201A6843291CA0
:106260000138FAF765F980B238BDC046D800002081
:10627000E703000000000000000000000000000034
:1062800008B56420FBF704FB00BE08BD0000000059
:10629000F0B51F2357464E4645469A46E0B4804621
:1062A0000027012682B0381CFEF742F83F23051C68
:1062B0000024994602E00134092C22D02B1C2341F2
:1062C000E2B21E42F7D001AB1A705F700020019954
:1062D000FFF73EFC83B243450CD003041B0E1A1C8F
:1062E00051468A4349468B4301D0A02AE3D1C0B22C
:1062F0004045E0D1012002B01CBC90469946A24620
:10630000F0BD0137FFB2092FCDD10020F3E7C04621
:1063100010B5041C2C20FFF7BBFF002802D0201C66
:10632000FFF7B6FF10BDC0460000000000000000EF
:1063300010B500F0EDFA002800D116E1B848FFF7DB
:1063400017FF6424013CFDF7DBFEE4B20A20FBF7F3
:106350009FFA002CF6D1B348FFF70AFF2920FFF778
:10636000D7FF002800D010BD2A30FFF7D1FF00284A
:1063700000D004E10520FFF7CBFF002800D006E1A4
:10638000FFF7BEFC00F0D4FAA74C20700720FFF7FF
:10639000BFFF002800D0FDE0207800F0D1FA00F027
:1063A000E7FAA24C2070E020FFF7B2FF00280BD0E4
:1063B000012201202178CB07DB0F534003401A1C38
:1063C0000B1C8343134323703920FFF7A1FF0028E0
:1063D0000CD0012221788B07DB0F5A400123134098
:1063E0005A00022399430B1C13432370E220FFF74A
:1063F0008FFF00280CD0012221784B07DB0F5A4079
:10640000012313409A00042399430B1C1343237068
:10641000E620FFF77DFF00280CD0012221780B0732
:10642000DB0F5A4001231340DA00082399430B1C69
:1064300013432370E320FFF76BFF00280CD00122E9
:106440002178CB06DB0F5A40012313401A01102399
:1064500099430B1C134323703520FFF759FF002885
:106460000CD0012221788B06DB0F5A400123134008
:106470005A01202399430B1C134323703120FFF74B
:1064800047FF00280CD0012221784B06DB0F5A4031
:10649000012313409A01402399430B1C134323709B
:1064A0001120FFF735FF002808D001222178CB0901
:1064B0005340DA017F230B4013432370207800F010
:1064C0005FFA23785A4ADB0927201370FFF720FF71
:1064D000041C1E20FFF71CFF002802D002231C43CF
:1064E000E4B21F20FFF714FF002802D004231C434E
:1064F000E4B22020FFF70CFF002802D008231C4341
:10650000E4B22120FFF704FF002802D010231C432F
:10651000E4B22220FFF7FCFE002802D020231C4317
:10652000E4B22320FFF7F4FE00280ED040232420FD
:106530001C43E4B2FFF7ECFE00280BD1201C00F056
:106540000FFA201CFFF70CF80DE72420FFF7E0FE00
:1065500000280DD080235B421C43E4B2201C00F0D5
:10656000FFF9201CFEF7FCFFFDE600F0B9F9E5E6B7
:10657000002CE3D100F0ECF9FEF7F2FFF3E600F0B7
:10658000AFF90520FFF7C4FE002800D1F8E6FFF7B9
:1065900077FEF5E61B20FFF7BBFE00280DD0012299
:1065A00021788B07DB0F5A40012313405A00022346
:1065B00099430B1C13432370EEE60E20FFF7A8FE51
:1065C00000280DD0012221784B07DB0F5A40012310
:1065D00013409A00042399430B1C13432370DBE6FA
:1065E0001020FFF795FE217800280CD001220B0720
:1065F000DB0F5A4001231340DA00082399430B1C98
:1066000013432370C8E601220120CB07DB0F534060
:1066100003401A1C0B1C834313432370BCE6C04683
:10662000348800004C880000000C00200C0C002076
:1066300031FEFF1F0000000000000000000000000D
:106640000E4B10B51940C023DB0419430C4B1960E5
:106650000C4B1A6072B601230B4C0343201C984765
:1066600062B670222378134000D023708021074A3D
:10667000C900D3680B43D36010BDC046FCFFFF00C8
:10668000040002400800024000000240003000F018
:1066900070B5144C2268002A13D0FF267F2801D938
:1066A000301C70BD104B9A42FAD3FF2502E0023332
:1066B0009A42F5D32C1C19880C408442F7D10E0A5B
:1066C000F5E7094A094D0A4B02E002329A4205D227
:1066D0001188A942F9D1023A2260DEE79A1E2260AF
:1066E000DBE7C046100C002000F80000FFFF0000B0
:1066F0000000010000000000000000000000000099
:10670000F0B55F4656464D464446F0B4584BA7B0E8
:10671000041C0E1C02A857490E229B461D6801F05E
:1067200017F97F2C14D8291E00D18BE0524B9846C4
:106730000231414513D25B463202144319608B0784
:1067400000D47CE04D4A2404224302A8FFF778FFDE
:1067500027B03CBC90469946A246AB46F0BD06AD7C
:106760002B1CFF2226A91A7001338B42FBD144480F
:10677000804513D9FF22C14300239446A1464144DA
:106780004908013149006246C75A3A407F2A01D878
:106790003C0AAC5402338B42F5D14C462E55041CB6
:1067A000804527D9012302AA1A43364B061C9A4674
:1067B00090231B059946434680461C1C324F01928C
:1067C0004B4652463343136072B62F48019B98479D
:1067D00062B670223B78134000D03B708020C0002E
:1067E00084462A496644CA680243CA60B442E7D86C
:1067F00044461F1C022300269846AB5DFF2B06D0A3
:106800004246224211D11B0233431F1C023401367F
:10681000802EF2D15B461C60A30799D51C4A02A8C2
:106820003A43211CFFF70CFF92E7320417431B0683
:106830001F4302A8211C3A1CFFF702FFE6E7144A97
:10684000224382E70C4A0E4B0C49101C02E0023333
:10685000984207D91A888A42F9D1991E5B46804628
:10686000196065E75B46811E8046196060E7C04697
:10687000100C00207C7A000000000100FFFF0000E7
:1068800000F800000400024000000240003000F068
:106890000000FFFF000000000000000000000000FA
:1068A00038B5051CFFF7F4FE041C681CFFF7F0FE6A
:1068B00000020443A0B238BD000000000000000048
:1068C00038B5051C0C1CC9B2FFF71AFF681C210A59
:1068D000FFF716FF38BDC0460000000000000000B2
:1068E00008B500200949FFF7EBFF02200021FFF760
:1068F00007FF03200021FFF703FF04200021FFF71B
:10690000FFFE05200021FFF7FBFE08BDEDFE0000A5
:1069100008B50020FFF7C4FF034B9C466044434288
:106920005841C0B208BDC0461301FFFF000000007F
:1069300008B50220FFF7ACFE08BDC046000000000D
:1069400008B5011C0220FFF7DBFE08BD00000000B7
:1069500008B50320FFF79CFE08BDC04600000000FC
:1069600008B5011C0320FFF7CBFE08BD00000000A6
:1069700008B50420FFF78CFE08BDC04600000000EB
:1069800008B5011C0420FFF7BBFE08BD0000000095
:1069900008B51A4B1B78DA0708D5194B1B789800F5
:1069A000C3189B087F207F2B0AD908BD9A070CD5F6
:1069B000134B1B789800C3185B087F207F2BF4D8FB
:1069C0007E38002BF1D0D8B2EFE75B0708D40D4B2F
:1069D00005201B78002BE8D00B4A11788B4204D39A
:1069E000074B18788300C318DCE7054A127890003B
:1069F00080185843F9F72CFE83B2D3E7140C00201B
:106A000039FEFF1F1D0C00203AFEFF1F0000000092
:106A100008B5164B1B78DA0707D5154B1B789B0872
:106A20000120002B00D0D8B208BD9A0703D5104B27
:106A30001B785B08F4E75B0705D50D4B1B787F20BF
:106A40007F2BF1D8ECE70B4B1B78002B0AD00A4ABE
:106A500011788B42F1D2064A10785843F9F7F8FDC5
:106A600083B2ECE70123D8B2DEE7C046140C002065
:106A70003CFEFF1F1D0C002038FEFF1F0000000021
:106A800008B5F02828D0F1282CD0F2282FD0F328F0
:106A90001DD0F92831D0FA2834D0FB2838D0FC2872
:106AA0003CD0F42845D0F52849D0F6284DD0F72819
:106AB00051D0F82855D0FD2835D0FE2857D0FF28D2
:106AC00009D104232D4A11780B43137003E0FFF71B
:106AD0005FFF2B4B587008BDFFF75AFF284B404211
:106AE0009870F8E7FFF754FF254B9870F3E7FFF72E
:106AF0004FFF234B40425870EDE7FFF789FF204BD3
:106B0000D870E8E7FFF784FF1D4B4042D870E2E7FA
:106B1000FFF77EFF1A4B40421871DCE7FFF778FF62
:106B2000174B1871D7E70123144A11780B431370E0
:106B3000D1E70123124A11780B431370CBE70223EC
:106B40000F4A11780B431370C5E704230C4A1178E0
:106B50000B431370BFE70823094A11780B431370E6
:106B6000B9E71023064A11780B431370B3E70223E9
:106B7000024A11780B431370ADE7C046140C002095
:106B8000180C0020000000000000000000000000C1
:106B9000F02849D0F12835D0F2283FD0F32849D049
:106BA000F92800D16BE0FA2800D171E0FB2849D028
:106BB000FC284DD0F42854D0F52859D0F62800D11F
:106BC0007BE0F72800D17FE0F82800D183E0FD28A2
:106BD00064D0FE2800D185E0FF2800D166E0454B57
:106BE0005A78002A0DD102229A56002A09D103228E
:106BF0009A56002A05D11B795BB2002B01D13E4A7F
:106C00001370704702223B4B9A56002AE8DD00229F
:106C10009A7001229A56002AE9D0F2E7354B5A7849
:106C200051B20029DDDA0AE0324B9A787F2AEED899
:106C30005A78D6E72F4B5A7851B20029D1DD00227D
:106C40005A70D0E72B4B1A797F2A06D85A78C8E7B2
:106C50000422284B9A56002AC2DD00221A715A7863
:106C6000BFE70121234B1A788A431A705A78B8E794
:106C70000221204B1A788A431A705A78B1E703220E
:106C80001C4B9A56002AABDD0022DA705A78A8E72E
:106C9000184BDA787F2AF7D85A78A2E70121174AE9
:106CA00013788B431370134B5A789AE70421134AD5
:106CB00013788B4313700F4B92E704210D4B1A7816
:106CC0008A431A705A788CE708210A4B1A788A434B
:106CD0001A705A7885E71021064B1A788A431A7081
:106CE0005A787EE70221054A13788B431370014BD3
:106CF0005A7876E7180C00201D0C0020140C002098
:106D000070B5264B1B781B0708D4254C201CFDF7BB
:106D1000BFFBFFF74DFA234B188070BD2248FFF7E9
:106D200027FA1F4C21482178FFF722FA2048FFF765
:106D30001FFA01211F4D6156281CFFF719FA1E4E3C
:106D4000301CFFF715FA0221281C6156FFF710FAD4
:106D5000301CFFF70DFA0321281C6156FFF708FAD3
:106D6000301CFFF705FA0421281C6156FFF700FAD2
:106D70001248FFF7FDF9124D124B281C1978FFF746
:106D8000F7F91148FFF7F4F9104B281C1978FFF7B1
:106D9000EFF90F48FFF7ECF9B8E7C046000C002008
:106DA000180C00201E0C00205488000008870000EA
:106DB000788800007C88000004870000808800003C
:106DC000848800001D0C002088880000140C00201E
:106DD000BC8C00000000000000000000000000006B
:106DE000F0B5474680B44C4B82B01888FFF728FABC
:106DF0004A490A78002A68D0494B1B7883425BDCF9
:106E0000484C23796778A578E6789846002F57D1C3
:106E1000002D03D1002E01D1002B4DD0FF2A0BD025
:106E200001320A707BB2002B04DDFFF7B1FDC7B25F
:106E300067707BB2002B5ADB6DB2002D04DDFFF7CB
:106E4000A7FDC5B2A5706DB2002D49DB002F16D08D
:106E5000A578002D13D078B2F9F7CAFF324A334B28
:106E6000F9F7EEFCF9F78CFF607068B2F9F7C0FF34
:106E70002D4A2E4BF9F7E4FCF9F782FFA07073B2AC
:106E8000002B04DDFFF7C4FDC6B2E67073B2002B21
:106E900036DB6A4643460720D3711056002807DDCB
:106EA000FFF7B6FD6A46C3B207202371D3711056AF
:106EB000002810DBFFF724FF02B004BC9046F0BDB1
:106EC000FF2AAFD001320A70ACE7194B1B789C0047
:106ED000E3185B0092E7FFF79BFD40422071E9E772
:106EE000FFF756FD4042A070002FC8D0B0E7FFF773
:106EF0004FFD4042C7B26DB26770002D9FDCA3E723
:106F0000FFF786FD6A4640424346E0700720D37192
:106F100010560028C4DCCBE71E0C00201D0C0020FE
:106F20003DFEFF1F180C0020666666666666E63F3B
:106F30003BFEFF1F000000000000000000000000FA
:106F40000023044A13601371034A1370034A137039
:106F50007047C046180C00201D0C0020140C0020A7
:106F600008B50448FFF704F9034805210122FFF79B
:106F7000FFF808BDC48B0000C08C000000000000BA
:106F800008B506280DD82F4B80001B589F462E4B66
:106F90001A785118FE293CDCC9B219702B48FFF74A
:106FA000E7F808BD2A4A13785918FE2939DCC9B216
:106FB00011702848FFF7DCF8F3E7274A13785918CF
:106FC000FE2936DCC9B211702448FFF7D1F8E8E792
:106FD000234A13785918FE2927DCC9B211702148B9
:106FE000FFF7C6F8DDE7204A13785918FE2924DC9C
:106FF000C9B211701D48FFF7BBF8D2E71C4A1378DD
:107000005918FE2909DCC9B211701A48FFF7B0F807
:10701000C7E7FF22FF211A70C0E7FF23FF2113708B
:10702000F3E7FF23FF211370C3E7FF23FF21137052
:10703000D5E7FF23FF211370C6E7FF23FF2113705D
:10704000D8E7C0468C88000038FEFF1F7C8D00000A
:107050003BFEFF1F108D00003DFEFF1F208D000036
:107060003AFEFF1F488D000039FEFF1F348D0000DF
:107070003CFEFF1F608D00000000000000000000CB
:1070800008B506280DD82F4B80001B589F462E4A66
:10709000137899423DD2591AC9B211702B48FFF7A3
:1070A00067F808BD2A4A13788B423AD9591AC9B2EF
:1070B00011702848FFF75CF8F3E7274A13789942E4
:1070C00037D2591AC9B211702448FFF751F8E8E7CE
:1070D000234A1378994228D2591AC9B2117021480B
:1070E000FFF746F8DDE7204A1378994225D2591A6E
:1070F000C9B211701D48FFF73BF8D2E71C4A13785C
:1071000099420AD2591AC9B211701A48FFF730F8D9
:10711000C7E7002300211370C0E70023002113708C
:10712000F3E7002300211370C3E70023002113704D
:10713000D5E7002300211370C6E700230021137058
:10714000D8E7C046A888000038FEFF1F7C8D0000ED
:107150003BFEFF1F108D00003DFEFF1F208D000035
:107160003AFEFF1F488D000039FEFF1F348D0000DE
:107170003CFEFF1F608D00000000000000000000CA
:1071800010B5041C0548211CFEF7F2FF0120A040A9
:10719000FEF7E6F9FDF784FD10BDC046988D0000AE
:1071A000F8B5831FDBB2422B00D987E1D44A9B009C
:1071B000D3589F46FDF774FDD248FEF7D9FFFA2059
:1071C0008000FAF765FB0124FFF75AF8201CF8BD90
:1071D000F1230124CC4ACD4811780B40A34313700E
:1071E000FEF7C6FFCA48FEF7C3FFCA4B1C70EDE7A7
:1071F000C54D2C78E407E40FE4B2002C00D176E111
:10720000C548FEF7B5FFF0232A7813402B70DDE761
:10721000C248FEF7ADFFC248FEF7AAFFFFF798FB92
:10722000C04E011C301CFEF7A3FFBF4D281CFEF70B
:107230009FFFFFF77DFB041CBC48FEF799FFBC4F86
:10724000211C381CFEF794FF281CFEF791FFB9485B
:10725000FEF78EFFE107C90FC9B2301CFEF788FFA9
:10726000281CFEF785FFB448FEF782FFA107C90F6F
:10727000301CFEF77DFF281CFEF77AFFAF48FEF7B3
:1072800077FF6107C90F301CFEF772FF281CFEF75D
:107290006FFFAB48FEF76CFF2107C90F301CFEF7EC
:1072A00067FF281CFEF764FFFFF762FB041CA5487C
:1072B000FEF75EFF211C381CFEF75AFF281CFEF764
:1072C00057FFA148FEF754FFE107C90FC9B2301CB0
:1072D000FEF74EFF281CFEF74BFF9C48FEF748FFC9
:1072E000A107C90F301CFEF743FF281CFEF740FF23
:1072F0009748FEF73DFF6107C90F301CFEF738FFC6
:10730000281CFEF735FF9348FEF732FF2107C90F0F
:10731000301CFEF72DFF281CFEF72AFF8E48FEF7D3
:1073200027FFE106C90F301CFEF722FF281CFEF7DD
:107330001FFF8A48FEF71CFFA106C90F301CFEF78D
:1073400017FF281CFEF714FF8548FEF711FF6106A2
:10735000C90F301CFEF70CFF281CFEF709FF8148FF
:10736000FEF706FF2106C90F301CFEF701FF281C9F
:10737000FEF7FEFE012429E77B48FEF7F9FE012413
:1073800024E701260421604D2B785C07E40F74404C
:10739000E4B2A2008B4313432B70002C00D1A1E078
:1073A0007248FEF7E5FE2B781E432E700EE701268D
:1073B0000821554D2B781C07E40F7440E4B2E2001D
:1073C0008B4313432B70002C00D186E06848FEF7F6
:1073D000CFFE2B781E432E70F8E6FDF761FC0122EC
:1073E000644B1C7854401C7072D06348FEF7C0FE9A
:1073F000ECE66248FEF7BCFEFCF7FAFF011C6048B1
:10740000FEF7B6FE5F4B60481978FEF7B1FE5F4BA2
:107410005F481978FEF7ACFE564B5E481978FEF7C8
:10742000A7FEFEF7EDFE011C5B48FEF7A1FE01245E
:10743000CCE65A48FEF79CFE5948FEF799FE59489B
:10744000FEF796FE5848FEF793FE5848FEF790FE6A
:107450005748FEF78DFE0124B8E6012602212A4D89
:107460002B789C07E40F7440E4B262008B43134313
:107470002B70002C27D04F48FEF77AFE2B781E4346
:107480002E70A3E64C48FEF773FE00F059FAFCF7A5
:10749000AFFFFCF78DFF012498E61D38C0B2FFF75F
:1074A0006FFE012492E60020FFF76AFE01248DE6BC
:1074B0003938C0B2FFF764FE012487E63F48FEF783
:1074C00057FE002482E63E48FEF752FE01247DE688
:1074D0003C48FEF74DFE012478E63B48FEF748FEA7
:1074E000012473E63948FEF743FE01246EE638486E
:1074F000FEF73EFE01232A78012413432B7065E634
:10750000C4880000A88F0000000C00207C8F0000C1
:10751000A48F0000200C0020BC8F0000B08D000064
:10752000BC8D000084880000F0910000CC8D00002C
:1075300008870000E08D0000EC8D0000F88D000051
:10754000048E0000108E0000248E0000408E00008B
:10755000588E00006C8E0000808E00008C8E000023
:10756000A08E0000BC8E0000C48E0000F88F0000CA
:107570001890000031FEFF1FC491000040910000F0
:107580005091000000FEFF1F6C910000F00A0020E7
:107590008491000098910000AC91000034900000AC
:1075A0004490000070900000B0900000E090000057
:1075B00034910000D88F0000A08D0000DC91000005
:1075C000E88F0000D0910000249000000890000097
:1075D000CC8F000000000000000000000000000050
:1075E00000207047000000000000000000000000C4
:1075F00000207047000000000000000000000000B4
:1076000070B57F4D061C2B78012B20D0002B0FD09E
:10761000022B08D1C31FDBB24B2B00D9DAE0794A29
:107620009B00D3589F46002300242B70201C70BD64
:10763000754B00241B681B78222BF7D1FFF7D0FF76
:10764000041EF3D1301CFFF7ABFD041CEEE76E4BBC
:107650001B681B78222B0CD0FFF7CAFF041EE5D154
:107660000B3EF6B22D2E00D9B9E0684BB6009B59FF
:107670009F46FFF7B5FF041ED8D1E3E71E22644BF7
:1076800064481A70644B14321A70644B283A1A70AA
:10769000634B0A321A70634B0C3A1A70624B2032F9
:1076A0001A70FEF765FD614B1978002900D09AE049
:1076B0005F48FEF75DFD0124B8E7FFF751FC5B4B27
:1076C0001978F2E7594C0A212078FFF759FC217804
:1076D000EBE7564C0A212078FFF7D2FC2178E4E74B
:1076E000524C01212078FFF7CBFC2178DDE74F4C8D
:1076F00001212078FFF744FC2178D6E74B4B1A781C
:10770000002A75D000221A70D2E74A4B1E3EF6B20C
:10771000995D464B1970C8E74748FEF729FD474871
:10772000FEF726FD464D3A4B281C1978FEF720FD42
:10773000444C201CFEF71CFD4348FEF719FD364B58
:10774000281C1978FEF714FD201CFEF711FD3F4898
:10775000FEF70EFD314B281C1978FEF709FD201CA1
:10776000FEF706FD3A48FEF703FD2D4B281C19785D
:10777000FEF7FEFC201CFEF7FBFC3648FEF7F8FC8B
:10778000284B281C1978FEF7F3FC201CFEF7F0FCB0
:107790003148FEF7EDFC244B281C1978FEF7E8FC75
:1077A000201CFEF7E5FC214B19787EE700232B70A7
:1077B0003CE7FFF7D5FB2948FEF7DAFC022301245A
:1077C0002B7033E72648FEF7D3FC2648FEF7D0FCA3
:1077D00001242BE72448FEF7CBFC012426E72248AE
:1077E000FEF7C6FC22E72148FEF7C2FC01241DE794
:1077F0001C48FEF7BDFC012301242B7016E7C04690
:10780000200C0020D089000034FEFF1F008B0000F8
:107810003BFEFF1F709200003DFEFF1F39FEFF1F61
:107820003AFEFF1F3CFEFF1F38FEFF1F210C002009
:1078300088920000B88B0000E4910000F4910000F1
:1078400084880000F0910000089200001C92000063
:107850002C9200004092000058920000E09100003D
:107860007C8F0000A48F0000DC910000809200005B
:1078700038B57546F9F754FC124C23880133238040
:10788000DBB2002B10D062780F4992088A5C9A42D2
:1078900014D080230D4A11680B431360F9F758FC8C
:1078A000281CFAF705FB38BD0220FCF781FD627841
:1078B0000549920823788A5C9A42EAD10020FCF7B5
:1078C00077FDE6E7240C00208C92000000000440C5
:1078D00001230F490F4A10B588580F4C03438B50B2
:1078E000002301222360A3600C4B1C2059780A431B
:1078F0005A70022219780A431A70302302216360F9
:10790000FBF786F8402322681343236010BDC0466E
:1079100000700440381000000000044000400640A1
:107920000123024A11680B431360704700000440B2
:107930000121024A13688B43136070470000044022
:107940000123024A11684B40136070470000044055
:1079500070B50F2A32D9041C0C430B1CA40731D17B
:10796000151C041C103D2D0901352D0149191E68F7
:1079700026605E6866609E68A660DE681033E6601A
:1079800010349942F3D10F2345191340032B1BD90F
:107990001C1F0023A4080134A400CE58EE50043369
:1079A000A342FAD1ED18C91803231A4005D00023C9
:1079B000CC5CEC5401339342FAD170BD051C002A13
:1079C000F5D1FAE7051CF2E71A1CF8E70000000001
:1079D00070B583073FD0541E002A3BD0CEB2031CA3
:1079E000032503E0621E002C34D0141C01335A1E00
:1079F00016702B42F6D1032C24D9FF250D402A0204
:107A000015432A0415430F2C11D9261C103E3609A4
:107A1000013636011A1C9B19156055609560D560BA
:107A200010329342F8D10F221440032C0AD9261F9A
:107A3000B6080136B6001A1C9B1920C29342FCD12D
:107A400003221440002C05D0C9B21C19197001334F
:0C7A5000A342FBD170BD141C031CCCE74A
:107A5C002000000040000000800000000001000039
:107A6C0000020000000400000005000000060000F9
:107A7C008023037003785BB2002BFBDA70470000A5
:107A8C002C0A00000A0A00000A0A0000FE09000085
:107A9C00F2080000F2080000F2090000FE090000E4
:107AAC00F2080000F2090000F2080000FE090000D4
:107ABC00F6080000F6080000F60800000C0C0000A8
:107ACC000C930000280C0020280C0020280C00200F
:107ADC000C930000000000000000000000000000FB
:107AEC000C930000000000000000000000000000EB
:107AFC000C930000000000000000000000000000DB
:107B0C000C930000000000000000000000000000CA
:107B1C000C930000000000000000000000000000BA
:107B2C000C930000000000000000000000000000AA
:107B3C000C9300000000000000000000000000009A
:107B4C00647B000000000020D80000200100000031
:107B5C00410F00000000000069646C65000000002B
:107B6C00535623310000000053562332000000000E
:107B7C0053562333000000005356233400000000FA
:107B8C0053562335000000005356233600000000E6
:107B9C0053562337000000005356233800000000D2
:107BAC005356233900000000535623313000000097
:107BBC00535623313100000063685654446F5265AC
:107BCC00736574490000000063685654446F536534
:107BDC00744900005C1300005013000050130000A7
:107BEC0064130000461300003A1300005013000009
:107BFC004613000063685363685265616479416899
:107C0C006561644900000000636853636857616BE9
:107C1C006575705300000000737461636B206F76A0
:107C2C006572666C6F7700006368536368526561B8
:107C3C006479490063685468644372656174655380
:107C4C00757370656E646564490000006368546800
:107C5C00644372656174650063685468645375733A
:107C6C0070656E6453000000636854686452656C00
:107C7C006561736500000000636854686452657345
:107C8C00756D6549000000006368537973556E6C1F
:107C9C006F636B006368546864446F446571756509
:107CAC0075654E65787449006368546864536C65F7
:107CBC0065705300636854686445786974530000B8
:107CCC006D61696E00160020040444080C10141831
:107CDC001C202122230000006368537973556E6CBD
:107CEC006F636B0063685265674E65787454687295
:107CFC006561640063684D7478556E6C6F636B00DE
:107D0C0063684D74784F626A656374496E69740078
:107D1C006368537973556E6C6F636B0063684D7455
:107D2C00784C6F636B5300006368537973556E6CBA
:107D3C006F636B006368436F7265416C6C6F63417A
:107D4C006C69676E6564490063684865617046726A
:107D5C00656500006368537973556E6C6F636B00D7
:107D6C006368506F6F6C4672656549006F62714F46
:107D7C00626A656374496E697400000063685379C4
:107D8C0073556E6C6F636B006F627152656C6561DD
:107D9C007365456D7074794275666665724900004D
:107DAC006F6271476574456D70747942756666656E
:107DBC007254696D656F7574530000006F62715079
:107DCC006F737446756C6C42756666657253000011
:107DDC00C4280000F028000010290000C42800006E
:107DEC00C428000030290000CA2800009429000093
:107DFC009429000094290000E0290000C02900000B
:107E0C00942900009A290000757362496E697445C3
:107E1C006E64706F696E744900000000636853797A
:107E2C0073556E6C6F636B0075736244697361623A
:107E3C006C65456E64706F696E7473490000000068
:107E4C0075736253746172745265636569766549C2
:107E5C000000000000000000000000005F7573626D
:107E6C005F6570306F7574007573625374617274F2
:107E7C005472616E736D6974490000005F757362B2
:107E8C005F657030696E000001000000757362530D
:107E9C0074617274000000006E76696353657453EC
:107EAC00797374656D48616E646C65725072696F3C
:107EBC007269747900000000242C0000422C000030
:107ECC00242C0000382C00002E2C0000422C00002A
:107EDC00242C0000042C0000042C0000042C0000B6
:107EEC00042C0000042C0000042C0000042C0000C6
:107EFC00042C0000042C0000242C0000722C000028
:107F0C00682C00005E2C0000FC2B0000542C0000A0
:107F1C004A2C00005F70616C5F6C6C645F736574FD
:107F2C007061646D6F646500000000004125000005
:107F3C00B128000081290000400040008001002091
:107F4C000C0A002001000000040A002000F00F4081
:107F5C0016000000060000000600000016000000DD
:107F6C000100000001000000010000000100000001
:107F7C0001000000010000000100000001000000F1
:107F8C0001000000010000000100000001000000E1
:107F9C0001000000010000000500000005000000C9
:107FAC0001000000010000000100000001000000C1
:107FBC0001000000010000000100000001000000B1
:107FCC0001000000010000000100000001000000A1
:107FDC0040F00F4006000000060000000600000004
:107FEC00060000000100000001000000010000007C
:107FFC000100000001000000010000000100000071
:10800C000100000001000000010000000100000060
:10801C00010000001200000012000000010000002E
:10802C000100000001000000010000000100000040
:10803C000100000001000000010000000100000030
:10804C000100000001000000010000000100000020
:10805C000100000080F00F40060000000600000048
:10806C0006000000060000000600000006000000EC
:10807C0006000000060000000100000001000000E6
:10808C0001000000010000000100000001000000E0
:10809C0001000000010000000100000001000000D0
:1080AC0001000000010000000100000001000000C0
:1080BC0001000000010000000100000001000000B0
:1080CC0001000000010000000100000001000000A0
:1080DC000100000001000000C0F00F40060000008D
:1080EC00060000000600000006000000060000006C
:1080FC000600000006000000060000000100000061
:10810C00010000000100000001000000010000005F
:10811C00010000000100000001000000010000004F
:10812C00010000000100000001000000010000003F
:10813C00010000000100000001000000010000002F
:10814C00010000000100000001000000010000001F
:10815C0001000000010000000100000000F10F40D0
:10816C0001000000010000000100000001000000FF
:10817C0001000000010000000100000001000000EF
:10818C0001000000010000000100000001000000DF
:10819C0001000000010000000100000001000000CF
:1081AC0001000000010000000100000001000000BF
:1081BC0006000000060000000100000001000000A5
:1081CC00010000000100000001000000010000009F
:1081DC00010000000100000006000000010000008A
:1081EC00EC350000F035000018360000F4350000C6
:1081FC00EC350000EC350000EC350000EC350000EF
:10820C00EC350000EC350000EC350000EC350000DE
:10821C00EC350000EC350000EC350000EC350000CE
:10822C00EC350000EC350000EC350000EC350000BE
:10823C00EC350000EC350000EC350000EC350000AE
:10824C00EC350000EC350000EC350000EC3500009E
:10825C00EC350000EC350000EC350000EC3500008E
:10826C00EC350000003600000C3600003036000003
:10827C0038360000403600003C3600003436000032
:10828C001C3600002C360000283600002436000076
:10829C0020360000FE390000C6390000BC39000051
:1082AC00D0390000FE390000090000007D84000078
:1082BC002203430068006900620069004F0053000C
:1082CC00200054004D004B0020007400650073002A
:1082DC0074000000090000007D84000005010906FF
:1082EC00A10175019508050719E029E7150025017D
:1082FC008102950575010508190129059102950161
:10830C007503910395787501150025010507190072
:10831C0029778102C000000040000000D0840000DA
:10832C0012000000CC830000D13A0000E1350000BF
:10833C00C13800009136000015000000E0830000F9
:10834C0086000000208400000300000000000000F4
:10835C00D13600000000000008000000C40A002014
:10836C0000000000020000000000000005010902EE
:10837C00A1010901A1000509190129051500250113
:10838C00750195058102750395018103050109307D
:10839C0009311581257F75089502810609381581EB
:1083AC00257F35004500750895018106050C0A38B6
:1083BC00021581257F750895018106C0C00000005B
:1083CC001201000200000040EDFE0C0A0A0001023E
:1083DC00030100000631FF0974A15375081500262E
:1083EC00FF00951009758102C00000000403090408
:1083FC000300000000000000C13600000000000077
:10840C00080000009C0A0020000000000200000090
:10841C000000000009028600050100A032090400DA
:10842C000001030101000921110100012240000794
:10843C0005810308000A090401000103000000097A
:10844C0021110100012251000705820308000109D6
:10845C000402000103000000092111010001221592
:10846C000007058303100001090403000103000049
:10847C0000092111010001223100070584030800C5
:10848C000A09040400010300000009211101000184
:10849C0022390007058503100001000009000000C7
:1084AC004B840000636F6E736F6C655F666C7573E5
:1084BC00685F6362000000006368537973556E6CEB
:1084CC006F636B0005010906A1017501950805078D
:1084DC0019E029E715002501810295017508810332
:1084EC00950575010508190129059102950175037A
:1084FC00910395067508150026FF0005071900293C
:10850C00FF8100C0030000000000000021370000C4
:10851C000000000010000000400B002000000000D4
:10852C00020000000000000003000000000000003A
:10853C00A13600000000000008000000840A0020A2
:10854C000000000002000000000000000400000019
:10855C00F88300000C000000F085000022000000F1
:10856C00BC8200001600000004FEFF1F510000003A
:10857C007883000005010980A1018502150126B749
:10858C0000190129B7751095018100C0050C09016E
:10859C00A10185031501269C0219012A9C02751064
:1085AC0095018100C00000000900000064840000F7
:1085BC000300000000000000B136000000000000C5
:1085CC0010000000B00A00200000000002000000B3
:1085DC000000000031000000808500000900000050
:1085EC00328400000C0354004D004B002000C600E8
:1085FC0039000000E882000055534220636F6E661C
:10860C006967757265642E0A000000004B6579621B
:10861C006F6172642073746172742E0A0000000022
:10862C005B735D00F1A10000291E1F202122232471
:10863C002526272D2E2A2A2B141A0815171C180C40
:10864C0012132F30314C39041607090A0B0D0E0F7B
:10865C00333428284BE11D1B061905111036373809
:10866C00E5E5524EE0E3E2652C2C2C2CC0E6E7E469
:10867C0050514F000000000000353A3B3C3D3E3F5E
:10868C004041424344452A2A0101010101010101F3
:10869C0001010101010101010101010101010101BE
:1086AC0001010101010101010101010101010101AE
:1086BC00010101010101010101010101010101019E
:1086CC000101010100000000000000007A420000DE
:1086DC006842000056420000904200008C420000AC
:1086EC00A2420000444200002E410000B4420000AF
:1086FC00626F756E6365213A200000002530325898
:10870C00000000000A722F632030313233343536CA
:10871C003738394142434445460A0000253031364A
:10872C00620000006B6579626F6172645F726570E4
:10873C006F72743A2000000025303258200000007F
:10874C004C45443A20253032580A0000D6490000E6
:10875C00D6490000FC490000FC490000404A0000DA
:10876C005A4A0000BC490000BC4900006A4A00009B
:10877C00BC490000AE4A0000AE4A0000C4490000EB
:10878C00BC490000BC490000C44A0000044B000076
:10879C00044B0000044B0000044B0000044B000091
:1087AC00044B0000044B0000044B0000044B000081
:1087BC00044B0000044B0000044B0000044B000071
:1087CC00044B0000044B0000044B0000EE4A000078
:1087DC00E04A0000D24A0000244B00006164645F50
:1087EC006B65795F6269743A2063616E27742061EE
:1087FC0064643A20253032580A00000064656C5FCE
:10880C006B65795F6269743A2063616E27742064CA
:10881C00656C3A20253032580A00000063685379A1
:10882C0073556E6C6F636B00626F6F746D6167690B
:10883C0063207363616E3A202E2E2E200000000000
:10884C00646F6E652E0A00006D6F7573656B6579CC
:10885C00205B62746E7C782079207620685D2872AB
:10886C0065702F61636C293A205B00007C0000006E
:10887C00256400005D280000257500002F00000015
:10888C00A26F0000A46F0000BA6F0000E66F00003A
:10889C00D06F0000FC6F00008E6F0000A270000013
:1088AC00A4700000BA700000E6700000D0700000E8
:1088BC00FC7000008E700000D0710000F0710000A0
:1088CC0010720000BC740000BC74000078730000CF
:1088DC00BC740000BC74000082730000BC74000007
:1088EC00AE730000DA730000BC740000BC740000AE
:1088FC00BC740000BC740000F2730000BC74000077
:10890C00BC74000032740000BC7400005A74000087
:10891C00BC740000847400009A7400009A74000007
:10892C009A7400009A7400009A7400009A74000003
:10893C009A7400009A7400009A740000A6740000E7
:10894C00BC740000A6740000BC740000BC74000071
:10895C00BC740000BC740000BC740000BC7400004B
:10896C00BC740000BC740000BC740000BC7400003B
:10897C00BC740000A6740000BC740000BC74000041
:10898C0078730000BC740000B0740000B074000078
:10899C00B0740000B0740000B0740000B07400003B
:1089AC00B0740000B0740000B0740000A674000035
:1089BC00BC740000BC740000BC740000BC740000EB
:1089CC00B47100007C760000D4770000D4770000EE
:1089DC00D4770000BA760000D4770000D47700007A
:1089EC00D4770000D4770000D4770000D47700004F
:1089FC00D477000018770000FC760000D4770000D4
:108A0C00D4770000D4770000D4770000D47700002E
:108A1C00D4770000D4770000D4770000D47700001E
:108A2C000A7700000A7700000A7700000A77000036
:108A3C000A7700000A770000D4770000D477000092
:108A4C00D4770000D4770000D4770000FC760000C7
:108A5C00D4770000D4770000D4770000D4770000DE
:108A6C00D4770000D4770000D4770000D4770000CE
:108A7C00D4770000D4770000D4770000D4770000BE
:108A8C00D4770000D4770000BA760000D4770000C9
:108A9C00D4770000D4770000D4770000D47700009E
:108AAC00D4770000D4770000D4770000D47700008E
:108ABC00D4770000D4770000D4770000D47700007E
:108ACC00D4770000D4770000D4770000D47700006E
:108ADC00D4770000C4760000D4770000D47700006F
:108AEC00D2760000D4770000D4770000E076000046
:108AFC00EE760000C4770000DE770000DE77000021
:108B0C00DE770000DE770000B2770000DE77000031
:108B1C00DE770000DE770000AC770000DE77000027
:108B2C00DE770000DE770000DE770000DE770000E5
:108B3C00DE770000DE770000DE770000DE770000D5
:108B4C00DE770000DE770000DE770000DE770000C5
:108B5C00DE770000DE770000DE770000DE770000B5
:108B6C00DE770000DE770000DE770000AC770000D7
:108B7C00DE770000DE770000DE770000DE77000095
:108B8C00DE770000DE770000DE770000DE77000085
:108B9C00DE770000DE770000DE770000DE77000075
:108BAC00DE770000DE770000C477000001020304CA
:108BBC0005060708090000000A092D204D6F757382
:108BCC00656B6579202D0A4553432F713A097175F0
:108BDC0069740A313A0964656C6179282A31306DFF
:108BEC0073290A323A09696E74657276616C286D64
:108BFC0073290A333A096D61785F73706565640A8D
:108C0C00343A0974696D655F746F5F6D61780A350C
:108C1C003A09776865656C5F6D61785F737065653F
:108C2C00640A363A09776865656C5F74696D655FCF
:108C3C00746F5F6D61780A0A703A097072696E74AC
:108C4C002076616C7565730A643A097365742064E7
:108C5C00656661756C74730A75703A092B310A6418
:108C6C006F776E3A092D310A706775703A092B319E
:108C7C00300A7067646F776E3A092D31300A0A73C7
:108C8C0070656564203D2064656C7461202A206DDC
:108C9C0061785F7370656564202A20287265706541
:108CAC006174202F2074696D655F746F5F6D6178DE
:108CBC00290A000077686572652064656C74613AF6
:108CCC0020637572736F723D25642C20776865651F
:108CDC006C3D25640A53656520687474703A2F2FB7
:108CEC00656E2E77696B6970656469612E6F72674A
:108CFC002F77696B692F4D6F7573655F6B65797332
:108D0C000A0000006D6B5F64656C6179203D202565
:108D1C00640A00006D6B5F696E74657276616C201D
:108D2C003D2025640A0000006D6B5F6D61785F73F8
:108D3C0070656564203D2025640A00006D6B5F74CE
:108D4C00696D655F746F5F6D6178203D2025640AE5
:108D5C00000000006D6B5F776865656C5F6D617816
:108D6C005F7370656564203D2025640A0000000077
:108D7C006D6B5F776865656C5F74696D655F746F4B
:108D8C005F6D6178203D2025640A00004C25640A43
:108D9C0000000000536C656570204C4544207465E0
:108DAC0073740A006565636F6E6669673A0A000042
:108DBC0064656661756C745F6C617965723A2000EC
:108DCC0064656275675F636F6E6669672E72617743
:108DDC003A2000002E656E61626C653A200000003E
:108DEC002E6D61747269783A200000002E6B6579E3
:108DFC00626F6172643A20002E6D6F7573653A2054
:108E0C00000000006B65796D61705F636F6E666961
:108E1C00672E7261773A20002E737761705F636FF3
:108E2C006E74726F6C5F636170736C6F636B3A20FE
:108E3C00000000002E636170736C6F636B5F746F66
:108E4C005F636F6E74726F6C3A2000002E737761E3
:108E5C00705F6C616C745F6C6775693A2000000020
:108E6C002E737761705F72616C745F726775693AAB
:108E7C00200000002E6E6F5F6775693A20000000BD
:108E8C002E737761705F67726176655F6573633AA5
:108E9C00200000002E737761705F6261636B736CEE
:108EAC006173685F6261636B73706163653A200024
:108EBC002E6E6B726F3A20000A092D204D61676986
:108ECC0063202D0A643A0964656275670A783A0969
:108EDC006465627567206D61747269780A6B3A0912
:108EEC006465627567206B6579626F6172640A6D87
:108EFC003A096465627567206D6F7573650A763A19
:108F0C000976657273696F6E0A733A0973746174CA
:108F1C0075730A633A09636F6E736F6C65206D6FBE
:108F2C0064650A302D343A096C61796572302D34E0
:108F3C00284631302D4634290A506175733A09623E
:108F4C006F6F746C6F616465720A653A0965657060
:108F5C00726F6D0A6E3A094E4B524F0A7A3A097388
:108F6C006C656570204C454420746573740A000070
:108F7C000A092D20436F6E736F6C65202D0A4553C3
:108F8C00432F713A09717569740A6D3A096D6F75E1
:108F9C0073656B65790A0000433E20000A0A626F14
:108FAC006F746C6F616465722E2E2E2000000000B1
:108FBC000A64656275673A206F66660A00000000F5
:108FCC000A64656275673A206F6E0A000A6D6174F7
:108FDC007269783A206F6E0A000000000A6D6174A5
:108FEC007269783A206F66660A0000000A6B657930
:108FFC00626F6172643A206F6E0A00000A6B6579C9
:10900C00626F6172643A206F66660A000A6D6F7552
:10901C0073653A206F6E0A000A6D6F7573653A209E
:10902C006F66660A000000000A092D2056657273EF
:10903C00696F6E202D0A0000444553433A20225498
:10904C004D4B206B6579626F617264206669726D3D
:10905C0077617265206F7665722043686962694F2B
:10906C0053220A005649443A203078464545442854
:10907C0022544D4B2229205049443A20307830411B
:10908C003043282243686962694F5320544D4B206A
:10909C00746573742229205645523A20307830304A
:1090AC0030410A004255494C443A206637666162A9
:1090BC0064362D6469727479202830393A30343A28
:1090CC003233204F63742020312032303136290A5C
:1090DC00000000004F5054494F4E533A204348492A
:1090EC0042494F5320424F4F544D41474943204D25
:1090FC004F5553454B45592045585452414B4559B2
:10910C0020434F4E534F4C4520434F4D4D414E4401
:10911C00204E4B524F20424F4F544C4F41444552DE
:10912C005F53495A450A00004743433A20342E39CD
:10913C002E3300000A092D20537461747573202D91
:10914C000A000000686F73745F6B6579626F6172FF
:10915C00645F6C65647328293A2025580A00000066
:10916C006B6579626F6172645F70726F746F636F3D
:10917C006C3A2025580A00006B6579626F61726445
:10918C005F69646C653A2025580A00006B6579624A
:10919C006F6172645F6E6B726F3A2025580A000023
:1091AC0074696D65725F72656164333228293A2087
:1091BC002530346C580A00004E4B524F3A206F6EDB
:1091CC000A0000004E4B524F3A206F66660A0000B0
:1091DC003F0000004D3E20000A092D2056616C75A1
:1091EC006573202D0A000000313A2064656C6179AA
:1091FC00282A31306D73293A20000000323A206958
:10920C006E74657276616C286D73293A20000000CB
:10921C00333A206D61785F73706565643A200000A5
:10922C00343A2074696D655F746F5F6D61783A20B4
:10923C0000000000353A20776865656C5F6D6178D9
:10924C005F73706565643A2000000000363A207741
:10925C006865656C5F74696D655F746F5F6D61786F
:10926C003A2000007365742064656661756C740A3D
:10927C00000000004D25643E200000004D3E000023
:10928C000000000000000000000000010204060ABB
:10929C000F17202C3A4A5D71879DB3C7DAE9F5FCAC
:1092AC00FFFCF5E9DAC7B39D87715D4A3A2C2017AC
:1092BC000F0A06040201000000000000000000007C
:1092CC000100000016033000780044004500410006
:1092DC00440042004500450046000000113C0000DF
:1092EC00213C0000113D0000A13D0000013E0000AA
:1092FC0005010000F00B0020280A141E08320000A3
:0400000300000411E4
:00000001FF
